:020000040800F2
:1000000020080020D5010008A9650008AB6500089C
:10001000AF650008B3650008B76500080000000080
:10002000000000000000000000000000BB650008A8
:10003000BD65000800000000BF650008ED01000874
:10004000EF010008EF010008EF010008EF010008D0
:10005000EF010008EF010008EF010008EF010008C0
:10006000EF010008EF010008EF010008EF010008B0
:10007000EF010008EF010008EF010008EF010008A0
:10008000EF010008EF010008EF010008EF01000890
:10009000EF010008EF010008EF010008EF01000880
:1000A000EF010008EF010008EF010008EF01000870
:1000B00009260008EF010008F1250008EF010008FB
:1000C000EF010008EF010008EF010008EF01000850
:1000D000EF010008CD1F00080D2C0008EF010008FB
:1000E000EF010008EF010008EF010008EF01000830
:1000F000EF010008EF010008EF010008EF01000820
:10010000EF010008EF010008EF010008EF0100080F
:10011000EF010008EF010008D3260008EF010008F6
:10012000EF010008EF010008EF010008EF010008EF
:1001300000F002F800F03FF80AA090E8000C8244BA
:100140008344AAF10107DA4501D100F034F8AFF297
:10015000090EBAE80F0013F0010F18BFFB1A43F0A5
:10016000010318476C8B00008C8B0000103A24BFF1
:1001700078C878C1FAD8520724BF30C830C144BF0C
:1001800004680C607047000000230024002500264E
:10019000103A28BF78C1FBD8520728BF30C148BFEA
:1001A0000B607047642906F07182002070471FB50C
:1001B0001FBD10B510BD06F029FC1146FFF7F7FF73
:1001C00006F0AAF906F047FC03B4FFF7F2FF03BC00
:1001D00001F0B4FE0948804709480047FEE7FEE702
:1001E000FEE7FEE7FEE7FEE7FEE7FEE7FEE7FEE7E7
:1001F00004480549054A064B70470000F302000811
:1002000031010008200200202008002020040020E6
:10021000200400200CB50020019000906C4800687C
:1002200040F480306A49086000BF6948006800F403
:10023000003000900198401C0190009818B9019876
:10024000B0F5A06FF1D16248006800F4003010B141
:100250000120009001E0002000900098012843D187
:100260005C48006840F010005A4908600846006881
:1002700020F0030008600846006840F002000860B3
:1002800053484068524948600846406848600846FC
:10029000406840F4806048600846406820F47C1064
:1002A00048600846406840F4E81048600846006826
:1002B00040F08070086000BF4548006800F00070A2
:1002C0000028F9D04248406820F0030040494860C7
:1002D0000846406840F00200486000BF3C48406863
:1002E00000F00C000828F9D10CBD10B5FFF792FF03
:1002F00010BD10B53648006840F001003449086070
:10030000084640683449084031494860084600685A
:10031000324908402E4908600846006820F48020D1
:1003200008600846406820F4FE0048604FF41F0053
:100330008860FFF7DAFF4FF000602949086010BDC0
:1003400010B5002100200022214B5B6803F00C0156
:1003500021B1042906D0082928D107E0214B224CDD
:10036000236027E01F4B204C236023E0184B5B6881
:1003700003F47010164B5B6803F48032022303EB26
:10038000904022B9194B4343174C23600DE0104BAA
:100390005B6803F4003323B1144B4343124C2360D6
:1003A00003E0104B4343104C236003E00D4B0E4C15
:1003B000236000BF00BF064B5B68C3F303130C4C04
:1003C000E15C094B1B68CB40074C236010BD00006B
:1003D00000100240002002400000FFF8FFFFF6FE80
:1003E00008ED00E000127A000000002000093D0046
:1003F0000400002031490143314A1160704770B553
:10040000002100230F22C47804B32D4C246804F487
:10041000E064C4F5E064210AC1F10403CA404478F1
:1004200004FA03F18478144021430901254C06782D
:10043000A155047804F01F050124AC4005786D1126
:10044000AD0005F1E025C5F8004109E0047804F0AD
:100450001F050124AC401C4D0678761145F8264056
:1004600070BD1A4A0A400243154B1B1F1A607047A1
:1004700039B1134A121D12680243114B1B1D1A6039
:1004800006E00F4A121D126882430D4B1B1D1A60B5
:100490007047042808D14FF0E021096941F00401B8
:1004A0004FF0E022116107E04FF0E021096921F0EF
:1004B00004014FF0E0221161704700000000FA05CE
:1004C0000CED00E000E400E080E100E080FFFF1FB1
:1004D00010B50446CC48844208D10121042000F024
:1004E0002DFB0021042000F029FB46E0C748844290
:1004F00008D10121082000F021FB0021082000F094
:100500001DFB3AE0C248844208D10121102000F0CE
:1005100015FB0021102000F011FB2EE0BD488442A5
:1005200008D10121202000F009FB0021202000F04B
:1005300005FB22E0B848844208D10121402000F0A8
:10054000FDFA0021402000F0F9FA16E0B348844299
:1005500008D10121802000F0F1FA0021802000F074
:10056000EDFA0AE0AE48844207D10121801500F07F
:10057000E5FA0021A01500F0E1FA10BD10B5012147
:10058000084600F0DBFA0021012000F0D7FA10BD88
:100590002DE9F0410246002500260020002300241A
:1005A000002791F803C00CF00F0591F803C00CF080
:1005B000100CBCF1000F03D091F802C04CEA050505
:1005C00091F800C0BCF1000F31D0146800202BE07E
:1005D0004FF0010C0CFA00F3B1F800C00CEA03066E
:1005E0009E4220D183004FF00F0C0CFA03F7BC435E
:1005F00005FA03FC4CEA040491F803C0BCF1280F8F
:1006000006D14FF0010C0CFA00FCC2F814C00AE04D
:1006100091F803C0BCF1480F05D14FF0010C0CFA62
:1006200000FCC2F810C0401C0828D1D31460B1F8F7
:1006300000C0BCF1FF0F34DD546800202EE000F153
:10064000080C4FF0010808FA0CF3B1F800C00CEAEE
:1006500003069E4221D183004FF00F0C0CFA03F7E2
:10066000BC4305FA03FC4CEA040491F803C0BCF156
:10067000280F05D100F1080C08FA0CF8C2F8148014
:1006800091F803C0BCF1480F07D100F1080C4FF0FE
:10069000010808FA0CF8C2F81080401C0828CED3D4
:1006A0005460BDE8F0814FF6FF7101800221817036
:1006B0000421C17070470246002093680B400BB1C3
:1006C000012000E0002070470146886880B2704732
:1006D00002460020D3680B400BB1012000E000204F
:1006E00070470146C86880B2704701617047416138
:1006F00070470AB1016100E041617047C160704715
:100700004FF480320A438261816182618269826929
:10071000704702460020434B18684FF6807318401C
:1007200040EA021008433F4B186070473E49C861D9
:100730007047F0B50A46002300240021002500F090
:100740000046B6F1004F02D1364EF16901E0354E58
:100750007168C0F3034583B200F44016B6F5401F3C
:1007600008D121F070612F4E766826F070662D4F0B
:100770007E6012E000F48016B6F5801F06D10326D5
:1007800006FA05F4A14341F0706106E0460D36011A
:1007900003FA06F6B14341F0706122B1460D36010D
:1007A00003FA06F6314300F00046B6F1004F02D1DD
:1007B0001C4EF16101E01B4E7160F0BD30B50022AE
:1007C0008B071C0F0F2303FA04F2164B08338C100F
:1007D00053F824309343134C08348D1044F82530DB
:1007E00023468C1053F824308C07240F00FA04F4AD
:1007F00023430C4C08348D1044F8253030BD0A4991
:10080000DC3108607047000000080140000C014026
:10081000001001400014014000180140001C01407C
:10082000002001400000014000002042DF48006835
:1008300040F00100DD49086008464068DC49084096
:10084000DA49486008460068DA490840D749086034
:100850000846006820F4802008600846406820F4BC
:10086000FE0048604FF41F0088607047CF49096858
:1008700021F48031CD4A11601146096821F48021AC
:100880001160B0F5803F03D0B0F5802F0ED106E0A7
:10089000C649096841F48031C44A116007E0C34980
:1008A000096841F4A021C14A116000E000BF00BF07
:1008B000704710B501460022002300204A11012A8A
:1008C00002D1BA4C236806E0022A02D1B74C236A4F
:1008D00001E0B64C636A01F01F02012494401C4001
:1008E0000CB1012000E0002010BD38B500200090C0
:1008F0000024002500BF3120FFF7DBFF05460098EC
:10090000401C00900098B0F5A06F01D0002DF2D0EF
:100910003120FFF7CEFF08B1012400E0002420467B
:1009200038BD01460020A14A106820F0F80040EAD6
:10093000C10010607047A04908607047024600205F
:100940009A4B586820F47C1042EA01031843974BF5
:100950005860704798490866704701460020934ADE
:10096000506820F003000843506070478F4840688B
:1009700000F00C007047014600208C4A506820F0BF
:10098000F00008435060704701460020874A5068D5
:1009900020F4E06008435060704701460020834A1D
:1009A000506820F4605040EAC1005060704729B19F
:1009B0007E4A527A02437D4B5A7204E07B4A527A55
:1009C00082437A4B5A7270477B49D831086070472E
:1009D00001460020754A506820F4404008435060AA
:1009E00070470021714A20321170704A82F820103D
:1009F000012802D004280AD104E001216B4A2032E8
:100A0000117005E00521694A2032117000E000BF35
:100A100000BF70476949086070476449096A01432B
:100A2000624A11627047654944390860704730B5C1
:100A300000210022002400235C4D6D6805F00C01AC
:100A400021B1042905D0082923D105E05C4D0560BA
:100A500022E05B4D05601FE0544D6D6805F4701297
:100A6000524D6D6805F48034022505EB92421CB9A5
:100A7000544D554305600BE04C4D6D6805F4003551
:100A80001DB1504D5543056002E04D4D5543056085
:100A900002E04B4D056000BF00BF444D6D6805F09E
:100AA000F0010909484D6B5C0568DD4045603F4D2C
:100AB0006D6805F4E061090A434D6B5C4568DD40F3
:100AC00085603A4D6D6805F46051C90A3E4D6B5C16
:100AD0004568DD40C560354D6D6805F44041890BC2
:100AE0003A4D6B5CC568B5FBF3F5056130BD29B1C6
:100AF0002E4A526902432D4B5A6104E02B4A526937
:100B000082432A4B5A61704729B1284A92690243AD
:100B1000264B9A6104E0254A92698243234B9A61ED
:100B2000704729B1214AD2690243204BDA6104E0BF
:100B30001E4AD26982431D4BDA61704729B11B4AB4
:100B4000D2680243194BDA6004E0184AD268824343
:100B5000164BDA60704729B1144A12690243134BED
:100B60001A6104E0114A12698243104B1A617047FE
:100B700012494039086070470F49C86470470B49F3
:100B8000C87170470948406A40F080700749486260
:100B9000704701460020054A92680A400AB10120C8
:100BA00000E0002070470149887270470010024041
:100BB0000000FFF8FFFFF6FE0000424280044242C0
:100BC00000127A0000093D001400002024000020DB
:100BD00010B50446FE48844208D10121C014FFF735
:100BE000ADFF0021E014FFF7A9FFC4E0B4F1804F8E
:100BF00008D101210846FFF7AEFF00210120FFF7D1
:100C0000AAFFB8E0F348844208D101210220FFF78F
:100C1000A2FF00210220FFF79EFFACE0EE488442D5
:100C200008D101210420FFF796FF00210420FFF7DF
:100C300092FFA0E0E948844208D101210820FFF793
:100C40008AFF00210820FFF786FF94E0E4488442F1
:100C500008D101211020FFF77EFF00211020FFF7AF
:100C60007AFF88E0DF48844208D101212020FFF785
:100C700072FF00212020FFF76EFF7CE0DA488442FB
:100C800008D101214014FFF759FF00216014FFF73C
:100C900055FF70E0D548844209D10121C804FFF70F
:100CA0004DFF00214FF40020FFF748FF63E0D048DC
:100CB000844209D101210805FFF740FF00214FF4CC
:100CC0008010FFF73BFF56E0CA48844209D101215A
:100CD0004805FFF733FF00214FF40010FFF72EFF08
:100CE00049E0C548844208D101214020FFF733FF85
:100CF00000214020FFF72FFF3DE0C048844208D18B
:100D000001218020FFF727FF00218020FFF723FF2C
:100D100031E0BB48844208D101218015FFF71BFF59
:100D20000021A015FFF717FF25E0B648844209D13E
:100D300001210804FFF702FF00214FF48030FFF784
:100D4000FDFE18E0B048844209D101214804FFF7B4
:100D5000F5FE00214FF40030FFF7F0FE0BE0AB484A
:100D6000844208D101218804FFF7E8FE00214FF4F6
:100D70008020FFF7E3FE10BD00220288944B9842CA
:100D80000ED0994B98420BD0B0F1804F08D0914BC8
:100D9000984205D0904B984202D0904B984204D193
:100DA0004FF68F731A404B881A438D4B984207D0E9
:100DB0008C4B984204D04FF6FF431A40CB881A431D
:100DC00002808B8883850B880385814B98420BD0EA
:100DD000854B984208D08B4B984205D08A4B98425D
:100DE00002D08A4B984201D10B7A03860123838279
:100DF000704770B5002400220023058C4FF6FE7664
:100E000035400584028C8388048B4FF68F752C4007
:100E1000B51E2C400D882C43751E2A400D892A438F
:100E20004D882A436A4DA8420BD06F4DA84208D086
:100E3000744DA84205D0744DA84202D0734DA8420B
:100E400013D14FF6F7752A404D892A434FF6FB75AB
:100E50002A408D882A434FF6FF652B404FF6FF55F9
:100E60002B408D892B43CD892B4383800483CD88F0
:100E70008586028470BD70B5002400220023058C95
:100E80004FF6EF7635400584028C8388048B48F654
:100E9000FF752C404FF6FF452C400D884FF6FF762E
:100EA00006EA05252C434FF6DF752A400D8906EA30
:100EB00005152A434D8806EA05152A43444DA842E4
:100EC00002D0494DA8421DD14FF67F752A404D8969
:100ED0004FF6FF7606EA05152A434FF6BF752A40FE
:100EE0008D8806EA05152A434FF6FF352B404FF251
:100EF000FF752B408D8906EA85052B43CD8906EACF
:100F000085052B4383800483CD880587028470BDCB
:100F100070B5002400220023058C4FF6FF66354093
:100F20000584028C8388848B4FF68F752C404FF696
:100F3000FC752C400D882C434FF6FF552A400D8937
:100F40004FF6FF7606EA05252A434D8806EA052571
:100F50002A431F4DA84202D0234DA8421DD14FF273
:100F6000FF752A404D894FF6FF7606EA05252A438C
:100F70004FF6FF352A408D8806EA05252A434EF6AE
:100F8000FF752B404DF6FF752B408D8906EA051540
:100F90002B43CD8906EA05152B4383808483CD88B6
:100FA0008587028470BD70B5002200230024058C63
:100FB0004EF6FF7635400584038C8488828B48F694
:100FC000FF752A404FF6FF452A400D8820E00000BB
:100FD000002C01400004004000080040000C0040CC
:100FE000001000400014004000340140004C01405B
:100FF000005001400054014000180040001C004017
:1010000000200040004001400044014000480140F1
:101010004FF6FF7606EA05252A434DF6FF752B406D
:101020000D8906EA05352B434D8806EA05352B4325
:10103000FA4DA84202D0FA4DA84208D14BF6FF75EE
:101040002C408D894FF6FF7606EA85152C43848067
:101050008283CD88A0F84050038470BD828B4FF20C
:10106000FF331A408283828B4FF6FF7303EA01231A
:101070001A4382837047F0B50C46154600220021C2
:101080000026078C4EF6FF7C07EA0C070784828B4C
:10109000018C4FF6FF7707EA043640F6FF473A40E7
:1010A0004FF6FF7707EA05273A434FF6FF7707EA3F
:1010B00003373A43D94FB8420ED0D94FB8420BD07C
:1010C000B0F1804F08D0D74FB84205D0D64FB842C4
:1010D00002D0D64FB84206D14DF6FF77394046F4DC
:1010E0008057394305E047F6FF57394044F48057AD
:1010F000394382830184F0BD828B4FF6F3731A402B
:101100008283828B0A4382837047F0B50C46154672
:10111000002200210026078C4FF6FF6C07EA0C071F
:101120000784828B018C4FF6FF7707EA04264FF67F
:101130000C773A404FF6FF7707EA03172F433A43FD
:10114000B64FB8420ED0B64FB8420BD0B0F1804F78
:1011500008D0B44FB84205D0B34FB84202D0B34F15
:10116000B84206D14FF6FF57394046F480773943ED
:1011700005E04FF2FF57394044F4807739438283CA
:101180000184F0BD028B4FF2FF331A400283028BC1
:101190004FF6FF7303EA01231A4302837047F0B549
:1011A0000C461546002200210026078C4FF6EF7CE6
:1011B00007EA0C070784028B018C4FF6FF7707EADA
:1011C000041640F6FF473A404FF6FF7707EA033729
:1011D0003A434FF6FF7707EA05273A438F4FB84265
:1011E0000ED08F4FB8420BD0B0F1804F08D08D4F4A
:1011F000B84205D08C4FB84202D08C4FB84206D1CD
:101200004FF6DF77394046F01007394305E04FF6D7
:101210005F77394044F01007394302830184F0BD01
:10122000028B4FF6F3731A400283028B0A43028348
:101230007047F0B50C46154600220021068C4FF68B
:10124000FE773E400684028B018C4FF60C763240CE
:101250007E1C06EA03162E433243704EB0420ED077
:101260006F4EB0420BD0B0F1804F08D06D4EB042FF
:1012700005D06D4EB04202D06C4EB04206D14FF652
:10128000FD76314044F00106314305E04FF6F57636
:10129000314044F00106314302830184F0BD70B552
:1012A00005460C465D4885420ED05D4885420BD010
:1012B000B5F1804F08D05B48854205D05A48854239
:1012C00002D05A48854200D100E000BF208850B9C2
:1012D0002389A28861882846FFF7ABFFE18828466A
:1012E000FFF79EFF25E0208804280AD12389A288E1
:1012F00061882846FFF753FFE1882846FFF742FF41
:1013000017E0208808280AD12389A2886188284606
:10131000FFF7FBFEE1882846FFF7EEFE09E0238990
:10132000A28861882846FFF7A6FEE1882846FFF7D5
:1013300095FE70BD2DE9F04105460C4600260127BB
:10134000608808B9022600E00026A088012801D1A3
:10135000022700E001272088A0B92389A28861889C
:101360002846FFF766FFE1882846FFF759FF2389E3
:101370003A4631462846FFF712FFE1882846FFF734
:1013800001FF13E02389A28861882846FFF707FF41
:10139000E1882846FFF7F6FE23893A46314628467B
:1013A000FFF747FFE1882846FFF73AFFBDE8F081E5
:1013B0000A884B881A438B881A43CB881A430B89B7
:1013C0001A434B891A438B891A43A0F8442070476B
:1013D0004FF6FF71818000210180C1804180017240
:1013E00070470021018041808180C180018141815D
:1013F0008181C1817047002101804180012181806C
:101400000021C180018170470021018041808180DD
:10141000C18001814181818170470000002C014021
:10142000003401400004004000080040000C00406F
:1014300021B1028842F00102028004E002884FF6E6
:10144000FE731A400280704731B1B0F8442042F474
:101450000042A0F8442005E0B0F84420C2F30E0298
:10146000A0F8442070471AB183890B43838102E0BE
:1014700083898B43838170478182704741EA0203ED
:10148000A0F8483070471AB183890B43838102E08A
:1014900083898B438381704701894FF6F87211402D
:1014A000018170470A46002101894FF68F73194068
:1014B00011430181704730B504460D462946204648
:1014C000FFF7F0FF208940F00700208130BD2DE9B3
:1014D000F04104460D4616461F46602D06D13B4698
:1014E000012231462046FFF75AFE05E03B46012225
:1014F00031462046FFF79DFE29462046FFF7D2FFE2
:10150000208940F007002081BDE8F08130B50C460D
:1015100000210189C9B24FF6FF7505EA032515437D
:1015200025432943018130BD2DE9F04105460E4692
:1015300017469846002443463A4631462846FFF768
:10154000E5FF2C894FF6F870044044F007044FF68D
:101550008F70044044F070042C81BDE8F081F0B538
:1015600004460D4616461F463B463246294620464F
:10157000FFF7CCFF208940F480402081F0BD018539
:10158000828270470A46002101884FF68F73194006
:10159000114301807047F0B50C4615461E460021E8
:1015A000002200230189028B038C4FF6F877394023
:1015B00021434FF6FC473A4040F201173A434FF6B9
:1015C000DD773B404FF6FF7707EA06172F433B4393
:1015D000018102830384F0BD0A460021018B4FF68E
:1015E0008F7319401143018370470A460021018B14
:1015F00048F6FF7319404FF6FF7303EA02231943BD
:10160000018370470A460021818B4FF68F73194082
:101610001143818370470A460021818B48F6FF738E
:1016200019404FF6FF7303EA022319438183704781
:1016300021B1028842F08002028004E002884FF665
:101640007F731A400280704721B1828842F0040201
:10165000828004E082884FF6FB731A4082807047D4
:1016600021B1828842F00802828004E082884FF62D
:10167000F7731A408280704721B1828842F00102DC
:10168000828004E082884FF6FE731A4082807047A1
:101690000A460021018B4FF6F7731940114301836D
:1016A00070470A460021018B4FF2FF7319404FF635
:1016B000FF7303EA02231943018370470A4600219E
:1016C000818B4FF6F77319401143818370470A46A7
:1016D0000021818B4FF2FF7319404FF6FF7303EA2D
:1016E00002231943818370470A460021018B4FF67C
:1016F000FB7319401143018370470A460021018B97
:101700004FF6FF3319404FF6FF7303EA02231943E4
:10171000018370470A460021818B4FF6FB73194005
:101720001143818370470A460021818B4FF6FF33B6
:1017300019404FF6FF7303EA022319438183704770
:101740000A460021018B4FF67F7319401143018334
:1017500070470A460021018BC1F30E014FF6FF735B
:1017600003EA02231943018370470A460021818B53
:101770004FF67F7319401143818370470A46002159
:10178000818BC1F30E014FF6FF7303EA0223194365
:10179000818370470A460021018C4FF6FD73194082
:1017A0001143018470470A460021018C4FF6F773FC
:1017B00019401143018470470A460021018C4FF6FD
:1017C000DF7319404FF6FF7303EA021319430184D4
:1017D00070470A460021018C4FF67F7319404FF67F
:1017E000FF7303EA02131943018470470A4600217C
:1017F000018C4FF6FF5319404FF6FF7303EA0223A3
:101800001943018470470A460021018C4FF2FF738F
:1018100019404FF6FF7303EA02231943018470470E
:101820000A460021018C4DF6FF7319404FF6FF73F5
:1018300003EA023319430184704730B500230124C1
:101840008C40A3B2048C9C430484048C02FA01F5FE
:10185000ADB22C43048430BD30B5002304248C4049
:10186000A3B2048C9C430484048C02FA01F5ADB24B
:101870002C43048430BD70B5034600200024184674
:10188000183001258D40ACB21D8CA5431D8409B1D3
:10189000082909D100EB6100056825F07005056095
:1018A0000568154305600EE00D1FC5F34E0528447D
:1018B000056825F4E045056005684FF6FF7606EA01
:1018C00002263543056070BD21B1028842F0020254
:1018D000028004E002884FF6FD731A4002807047D0
:1018E00021B1028842F00402028004E002884FF62F
:1018F000FB731A400280704721B1828842F0800257
:10190000828004E082884FF67F731A40828070479D
:1019100002884FF6F7731A40028002880A43028059
:10192000704782884FF68F731A40828082880A43FC
:101930008280704702894FF6F8731A40028102894B
:101940000A430281704702894FF67F731A40028171
:1019500002890A43028170478184704781857047FC
:10196000818670470187704781877047A0F84010D3
:10197000704702884FF6FF431A40028002880A43EC
:10198000028070470146888E70470146088F704775
:101990000146888F70470146B1F840007047014604
:1019A000888C70470146088D704702460020138AD4
:1019B0000B400BB1012000E000207047CA430282B7
:1019C000704730B50246002000230024158A05EA3E
:1019D0000103958905EA010413B10CB1012000E06F
:1019E000002030BDCA4302827047000010B5044693
:1019F000FB48844209D101218803FFF79FF80021A9
:101A00004FF48040FFF79AF832E0F648844209D15B
:101A100001214804FFF79FF800214FF40030FFF741
:101A20009AF825E0F048844209D101218804FFF7A3
:101A300092F800214FF48020FFF78DF818E0EB4872
:101A4000844209D10121C804FFF785F800214FF431
:101A50000020FFF780F80BE0E548844208D101211F
:101A60000805FFF778F800214FF48010FFF773F8AE
:101A700010BD2DE9F04786B005460E460024A2466B
:101A800000BFA1460027B08900B100BF2F462C8AB5
:101A90004CF6FF700440F08804432C82AC894EF66B
:101AA000F3100440B0883189084371890843044326
:101AB000AC81AC8A4FF6FF400440B0890443AC824D
:101AC00001A8FEF7B4FFC648874202D1DDF810A096
:101AD00001E0DDF80CA0A88900F4004040B10AEB59
:101AE000CA0000EB0A1031684900B0FBF1F807E0CA
:101AF0000AEBCA0000EB0A1031688900B0FBF1F86C
:101B00006420B8FBF0F004012009642101FB108976
:101B1000A88900F4004040B1322000EBC900B0FBBE
:101B2000F1F000F00700044308E0322000EB091058
:101B30006421B0FBF1F000F00F0004432C8106B0EB
:101B4000BDE8F0874FF41651016000218180C1800B
:101B500001810C21418100218181704710B502462D
:101B60000020108A4FF2FF0318400B884C88234353
:101B70008C882343CC8823431843108210BD002156
:101B8000018041808180C180704721B1828942F407
:101B90000052828104E082894DF6FF731A408281EF
:101BA0007047F0B50346002400260025002040F6CB
:101BB0006A17B94200D100BF1846C1F3421401F0C0
:101BC0001F06012707FA06F5012C01D10C3004E0AD
:101BD000022C01D1103000E014301AB107682F43F5
:101BE000076002E00768AF430760F0BD1AB1838A5F
:101BF0000B43838202E0838A8B4383827047028A8D
:101C00004FF6F0731A400282028A0A43028270473A
:101C100082894FF2FF731A40828182890A4382814E
:101C2000704721B1828942F00202828104E08289F8
:101C30004FF6FD731A4082817047028A4FF6DF73B8
:101C40001A400282028A0A430282704721B1028A44
:101C500042F48042028204E0028A4BF6FF731A408B
:101C600002827047C1F3080282807047014688886B
:101C7000C0F308007047818941F0010181817047FC
:101C8000028BD2B20283028B42EA012202837047A6
:101C9000028B02F47F420283028B0A430283704765
:101CA00021B1828A42F02002828204E0828A4FF6C9
:101CB000DF731A408282704721B1828A42F010029B
:101CC000828204E0828A4FF6EF731A408282704764
:101CD00021B1828A42F00802828204E0828A4FF6B1
:101CE000F7731A408282704721B1828942F4004220
:101CF000828103E08289C2F30E028281704721B1A2
:101D0000828A42F40062828204E0828A4FF2FF7388
:101D10001A4082827047828A4FF6FB731A40828291
:101D2000828A0A438282704721B1828A42F002028B
:101D3000828204E0828A4FF6FD731A4082827047E5
:101D400002460020B1F5007F00D100BF13880B4090
:101D50000BB1012000E00020704701F40072B2F5E1
:101D6000007F00D100BFCA430280704770B50246B1
:101D7000002400230025002040F66A16B14200D15D
:101D800000BFC1F3421501F01F03012606FA03F359
:101D9000012D02D19689334006E0022D02D1168A28
:101DA000334001E0968A33400C12012606FA04F40F
:101DB0001688344013B10CB1012000E0002070BD42
:101DC00010B50022002340F66A14A14200D100BFE2
:101DD0000A1201249440A3B2DC43048010BD000029
:101DE000003801400044004000480040004C0040E2
:101DF0000050004070B5482000F016F900F05EF881
:101E000000F028F84FF4E13000F05AF800F02CFF11
:101E1000002140F60F6000F069FA00F024FB47F261
:101E200030504FF08041888400F06CFB47F2305016
:101E3000064908806421084600F0BAFA4FF4FA75A2
:101E40002C4603480580001D048070BD2408004016
:101E50003C04004008B501211020FEF755FE4FF468
:101E60008070ADF8000010208DF8030003208DF87D
:101E7000020069460F48FEF78BFB08BD70B50446AB
:101E80000D480068401C0C490860A04210D14FF476
:101E900080710848FEF70FFCC0F10100C5B22A4668
:101EA0004FF480710348FEF724FC002002490860CB
:101EB00070BD0000001001402800002070470000A5
:101EC00010B586B00446012144F20400FEF71CFE62
:101ED0004FF40070ADF8140018208DF8170003209F
:101EE0008DF8160005A94B48FEF752FB4FF48060B1
:101EF000ADF8140004208DF8170005A94548FEF739
:101F000047FB01940020ADF80800ADF80A00ADF8D9
:101F10000C00ADF810000C20ADF80E0001A93E48F1
:101F2000FFF7A7FD012240F225513B48FFF739FE9C
:101F300001213948FFF729FE06B010BD00BF7047E8
:101F400000BF354A128802F04002002AF9D0C2B21E
:101F5000314B1B1D1A80704710B5044600BF20216D
:101F60002D48FFF7EDFE0028F9D02B48FFF77EFE45
:101F700010BD70B504460D4640212748FFF7EDFE21
:101F800080212548FFF71CFF13E021782248FFF746
:101F900069FE00BF40212048FFF7D2FE0128F9D199
:101FA00040211D48FFF7D9FE80211B48FFF708FF9D
:101FB000641C281EA5F10105E7D170BD0022174B56
:101FC0001A60174A1160174A1060704710B540F246
:101FD00025511148FFF7CAFED8B10F48FFF746FE5A
:101FE000C4B20F4800680D49096888420CD90D48F1
:101FF000006804700B480068401C0A4908600748E4
:102000000068401C0549086040F225510248FFF76E
:10201000D7FE10BD0008014000380140300000200C
:10202000340000202C00002010B504466FF004009E
:10203000FEF72FFAE11704EB5171C1F3C701234AF0
:1020400011701046007800EB4001C1EBC0104FF654
:10205000FF7101EAC0001E49088010BD01461C4AFC
:1020600012884A434FF0E0235A6100229A6101220C
:102070001A6100BF4FF0E022106900F001021AB1AE
:1020800000F48032002AF5D000224FF0E0231A61DC
:102090009A61704701460D4A12784A434FF0E02397
:1020A0005A6100229A6101221A6100BF4FF0E022BA
:1020B000106900F001021AB100F48032002AF5D054
:1020C00000224FF0E0231A619A6170473C00002023
:1020D0003E000020002001E0411CC8B20A28FBDBC2
:1020E000704710B54FF400617F48FEF7FEFA4FF4D9
:1020F00080617D48FEF7F9FAFFF7ECFF4FF40061CD
:102100007948FEF7F4FAFFF7E5FF4FF4806176486F
:10211000FEF7EDFAFFF7DEFF10BD10B54FF40061DA
:102120007148FEF7E4FA4FF480616F48FEF7DDFA7C
:10213000FFF7D0FF4FF400616B48FEF7D6FA10BDF1
:1021400070B50446002528E004F0800028B14FF463
:1021500000616548FEF7C9FA04E04FF40061624887
:10216000FEF7C5FAFFF7B6FF4FF480615E48FEF751
:10217000BCFAFFF7AFFF4FF480615B48FEF7B7FA98
:10218000072D04D14FF400615748FEF7AEFA600600
:10219000040EFFF79FFF681CC5B2082DD4DB70BD8D
:1021A00010B54FF400615048FEF7A1FAFFF792FF17
:1021B0004FF480614C48FEF798FAFFF78BFF4FF41D
:1021C00080614948FEF793FAFFF784FF4FF40061FE
:1021D0004548FEF78AFA10BD10B54FF40061424839
:1021E000FEF783FAFFF776FF4FF480613E48FEF773
:1021F0007CFAFFF76FFF4FF480613B48FEF777FAF8
:10220000FFF768FF10BD70B505460024002619E0F1
:102210006006040E4FF480613348FEF766FAFFF75C
:1022200059FF4FF400613048FEF745FA08B1601CD1
:10223000C4B24FF480612C48FEF759FAFFF74AFF09
:10224000701CC6B2082EE3DB15B9FFF7C5FF01E02D
:10225000FFF7A6FF204670BD10B54FF4006122487D
:10226000FEF743FAFFF736FF4FF480611E48FEF792
:102270003CFAFFF72FFF4FF400611B48FEF71BFAF3
:1022800008B1012400E000244FF480611648FEF7F5
:102290002EFAFFF71FFF204610BD08B501210820C8
:1022A000FEF732FC4FF44060ADF8000003208DF8DB
:1022B000020014208DF8030069460B48FEF768F908
:1022C000FFF72BFF08BD70B50446FFF7E6FFFFF7E9
:1022D00008FF2046FFF734FFFFF7BEFF0546FFF774
:1022E0001CFF284670BD0000000C014030B589B0CD
:1022F00005460C4601210220FEF713FC681E80B241
:10230000ADF80800A0B2ADF804000020ADF80A0056
:10231000ADF8060001A9C248FEF72EFD0121C04814
:10232000FFF74CFB01221146BD48FFF79CF8012145
:102330000820FEF7E9FB0320ADF8100018208DF807
:10234000130003208DF8120004A9B648FEF720F907
:102350006020ADF814000120ADF816000020ADF8A3
:102360001A00ADF81C0005A9AD48FEF7D1FD082103
:10237000AB48FFF73BFA6020ADF814000120ADF840
:1023800016000020ADF81A00ADF81C0005A9A448FD
:10239000FEF709FE0821A248FFF742FA0121A048F2
:1023A000FFF746F901219E48FFF742F809B030BD1A
:1023B0007FB505460C466020ADF800000120ADF861
:1023C0000200ADF8065069469548FEF7A1FD0821C8
:1023D0009348FFF70BFAADF8064069469048FEF7C0
:1023E000E2FD08218E48FFF71BFA01218C48FFF718
:1023F0001FF97FBD1FB501211020FEF792FB42F2AD
:102400000F70ADF8080040F2CF20ADF804000020B6
:10241000ADF80A00ADF806008DF80C0001A982485D
:10242000FEF7AAFC01218048FFF7C8FA01221146F5
:102430007D48FFF718F84FF44070FDF7DBFF3620BA
:102440008DF8000005208DF8010000208DF80200B5
:1024500001208DF803006846FDF7D1FF0121724885
:10246000FEF7E6FF1FBD00B587B001210846FEF765
:1024700058FB01210420FEF747FB0320ADF80000C4
:1024800004208DF8030069466848FEF781F804A827
:10249000FEF79EFF0020ADF810004EF66020ADF86C
:1024A00014004FF40070ADF816000020ADF81200D3
:1024B00004A94FF08040FEF75FFC00231A46032179
:1024C0004FF08040FFF767F801A8FEF794FF0A205D
:1024D000ADF80C0001A94007FEF7E1FE01218807D5
:1024E000FFF76CFA012211469007FEF7BCFF0021AE
:1024F0004FF08040FFF730FA01218807FEF798FF80
:1025000007B000BD00B587B001210420FEF709FB2C
:1025100001210820FEF7F8FAC020ADF800000420E1
:102520008DF8030069463F48FEF732F804A8FEF72D
:102530004FFF0020ADF810004EF66020ADF81400FB
:102540004FF40070ADF816000020ADF8120004A999
:102550003748FEF711FC00231A4603213448FFF7E1
:102560001AF801A8FEF747FF0A20ADF80C0001A9F0
:102570002F48FEF794FE01212D48FFF71FFA012294
:1025800011462B48FEF76FFF00212948FFF7E4F9B9
:1025900001212748FEF74CFF07B000BD0146022984
:1025A00004D003290CD004291ED113E04FF080423F
:1025B000928C10B247F230524FF080439A8415E06B
:1025C000174A2432128810B247F23052144B243387
:1025D0001A800BE0164A2432128810B247F23052A9
:1025E000134B24331A8001E0002000BF00BF704766
:1025F0000F48103000880E481030008820F001008D
:102600000B491031088070474FF08040008A4FF02E
:102610008040008A20F001004FF08041088270471E
:1026200000040040000C0140001000400008014080
:102630000008004003461846884200DD08469042E4
:1026400000DA1046704770B50546A049284605F0E7
:1026500077FA04D39E49284605F072FB01D2012483
:1026600000E00024204670BD2DE9FE4F04460D46D3
:10267000984E994F0021204605F093FB0290294681
:10268000002005F099FB01903946019805F08CFA7D
:1026900086F0004B00905846029905F085FA824674
:1026A000009905F089FB814605F0E2F98046404635
:1026B000BDE8FE8F10B501F043F8884800688849EE
:1026C00008608849B1F9000005F00EFA86490860F3
:1026D00010BD10B501218548FFF767F9002846D0E5
:1026E00001218248FFF77EF90520FFF7C7FB022092
:1026F000FFF754FF47F23051081A7D490860042063
:10270000FFF74CFF47F23051081A7A490860FFF78B
:10271000D1FF7548016872480068FFF7A5FF764948
:1027200008606F480068FFF78EFF10B100F014FBDF
:1027300010BD714800687149096808447049086013
:102740006D4800686D49096808446E4908606E4A22
:1027500051426B480068FFF76DFF694908606A4A9B
:10276000514268480068FFF765FF6649086000BF8E
:10277000DEE72DE9FF5F044689466448039064481C
:10278000029004EB0901484205F0AEF96149086086
:102790006148006804F0DCFF0746604A604B04F0C3
:1027A000E3FD054604F0A6FB5B4908605948006854
:1027B00004F0CEFF594A5B4BCDE9000104F0D4FD93
:1027C00005460E465448006804F0C2FF07462A46F4
:1027D000334604F0C1FB824604F08CFB4E4908608E
:1027E000084601685048006804F0DEFF4E49086062
:1027F0004E494D48006805F0A3FA02D24B484A49B9
:1028000008604B494848006805F09AF902D24848E8
:102810004549086044480299006805F0C5F9074633
:102820003D48006880F000463046039905F0BCF949
:102830000546394605F0C0FA3E4908602848006858
:10284000FFF701FF012803D03B480078012802D19F
:102850000020354908603748006805F009F904B0E0
:10286000BDE8F09F0146002901DA484200E0084631
:10287000704770B505460C46002D03DD002000F0C2
:1028800007FA02E0012000F003FA2846FFF7EAFF0A
:102890002A490880002C03DD002000F01BFA02E02A
:1028A000012000F017FA2046FFF7DCFF2349091D3D
:1028B000088070BD012807D11F49097809B9012195
:1028C00000E000211C4A117070470000000020C287
:1028D000000020420000C842713D8A3FC80000202D
:1028E00078000020B40000207C0000200010004090
:1028F00040000020440000208400002088000020C8
:102900008C0000209000002094F8FFFF000020437E
:10291000CDCC4C3F9C000020A00000209A999999B2
:102920009999E93F9999C93FA400002000401C46AD
:1029300000401CC698000020800000203C0400409D
:1029400010B586B0044601210420FEF7DDF8012110
:102950004804FEF7E6F80420ADF8140018208DF8BE
:10296000170003208DF8160005A9BA48FDF710FEE0
:102970000820ADF8140004208DF8170005A9B5480B
:10298000FDF706FE01940020ADF80800ADF80A003E
:10299000ADF80C00ADF810000C20ADF80E0001A948
:1029A000AD48FFF766F84FF4E060FDF723FD262001
:1029B0008DF8000000208DF801008DF80200012044
:1029C0008DF803006846FDF71AFD012240F22551FB
:1029D000A148FFF7E6F801219F48FFF7D6F806B0B7
:1029E00010BD70B504460D4640219B48FFF7B5F970
:1029F00080219948FFF7E4F913E021789648FFF722
:102A000031F900BF40219448FFF79AF90128F9D124
:102A100040219148FFF7A1F980218F48FFF7D0F9B5
:102A2000641C281EA5F10105E7D170BD10B5044650
:102A300040218948FFF791F980218748FFF7C0F9C5
:102A400013E014F8011B8448FFF70CF900BF402184
:102A50008148FFF775F90128F9D140217E48FFF739
:102A60007CF980217C48FFF7ABF920780028E8D179
:102A700010BDF0B503460D461646002729460A2E1E
:102A800003D0002008702846F0BD33B9302001F88B
:102A9000010B002008702846F6E7002B03DA2D20F2
:102AA00001F8010B5B4242F210720DE093FBF2F46D
:102AB00004B937B104F1300001F8010B04FB123303
:102AC00001270A2092FBF0F2002AEFDC00200870B8
:102AD0002846D9E70FB470B586B006460CA800901A
:102AE00040215D48FFF739F980215B48FFF768F91D
:102AF0007BE00B9800785C281CD10B98401C0B9055
:102B000000786E2809D072280FD10D213046FFF7CA
:102B1000A9F80B98401C0B900BE00A213046FFF7F8
:102B2000A1F80B98401C0B9003E00B98401C0B90F5
:102B300000BF4BE00B980078252840D10B98401C33
:102B40000B900078642818D0732833D1009810C8EF
:102B500000900BE021783046FFF784F800BF402159
:102B60003046FFF7EDF80028F9D0641C20780028E3
:102B7000F0D10B98401C0B9020E0009820C80090EA
:102B80000A2201A92846FFF774FF01AC0BE0217867
:102B90003046FFF767F800BF40213046FFF7D0F816
:102BA0000028F9D0641C20780028F0D10B98401C34
:102BB0000B9003E00B98401C0B9000BF06E00B98B5
:102BC00010F8011B0B903046FFF74CF800BF402176
:102BD0003046FFF7B5F80028F9D040211E48FFF72E
:102BE000BCF880211C48FFF7EBF80B980078002810
:102BF0007FF47FAF06B070BC5DF814FB0022174B6A
:102C00001A60174A1160174A1060704710B540F2F9
:102C100025511148FFF7AAF8D8B10F48FFF726F859
:102C2000C4B20F4800680D49096888420CD90D48A4
:102C3000006804700B480068401C0A490860074897
:102C40000068401C0549086040F225510248FFF722
:102C5000B7F810BD0008014000440040AC0000205F
:102C6000B0000020A800002008B501210820FDF7D1
:102C70004BFF4FF47C40ADF8000010208DF80300AE
:102C800003208DF8020069463748FDF781FC08BD36
:102C900010B504464CB94FF480513348FDF725FD7B
:102CA0004FF400513048FDF722FD012C07D161039C
:102CB0002D48FDF71AFD21032B48FDF718FD022CC6
:102CC00007D1E1022848FDF712FD21032648FDF750
:102CD0000EFD10BD10B504464CB94FF4004122481A
:102CE000FDF703FD4FF480411F48FDF700FD012C67
:102CF00007D1A1031C48FDF7F8FCE1031A48FDF7D2
:102D0000F6FC022C07D161031748FDF7F0FCA10384
:102D10001548FDF7ECFC10BD10B50020FFF7B8FF1B
:102D20000020FFF7D7FF10BD10B50120FFF7B0FF5F
:102D30000120FFF7CFFF10BD10B50120FFF7A8FF5E
:102D40000020FFF7C7FF10BD10B50020FFF7A0FF60
:102D50000120FFF7BFFF10BD10B50220FFF798FF5D
:102D60000220FFF7B7FF10BD000C014008B501219C
:102D70000820FDF7C9FE4FF44060ADF800001020B8
:102D80008DF8030003208DF802006946F748FDF72F
:102D9000FFFB08BD10B5F548001D006820F4704029
:102DA000F249091D08600846006840F44050086078
:102DB0000120EF490860EF48D0F82C0108B9002045
:102DC00010BD0120EA49091F0860FFF763F90020E0
:102DD000E849C1F8AC01E6488038006808B1002035
:102DE000EEE70120FFF756F90020E149091F0860CE
:102DF0000120E5E710B5DD48001D006820F47040B3
:102E0000DA49091D08600846006840F4405008602F
:102E10000020D749091F0860D649C1F8AC0101203C
:102E2000FFF738F90120D249091F0860D149C1F8DC
:102E3000AC01FFF72FF910BD10B50024CB48001DE1
:102E4000006820F47040C949091D08600846006800
:102E500040F4004008600120C5490860FFF71AF9F6
:102E60000120C449C1F8A801FFF714F90AE0601C69
:102E7000C4B2322C03DDFFF7BDFF002010BD0120DE
:102E8000FFF708F9BA48803800680028EFD1B84940
:102E9000091F08600120F1E710B50020B449091F9F
:102EA0000860B248001D006820F47040AF49091D59
:102EB00008600846006840F4405008600020AD49B2
:102EC000C1F8AC010120FFF7E5F80120A849091F6E
:102ED0000860FFF7DFF80020A649C1F8A80110BD7F
:102EE00010B50020A249091F0860A048001D006815
:102EF00020F470409D49091D08600846006840F4B0
:102F00004050086001209B49C1F8AC01FFF7C2F8AE
:102F100001209749091F0860FFF7BCF80020954978
:102F2000C1F8A80110BD70B504469048001D0068A6
:102F300020F470408D49091D08600846006840F47F
:102F40004050086000208A49091F0860002516E0EB
:102F5000E009874908606006040E0120FFF79AF82F
:102F600001208449C1F8A801FFF794F800208049A6
:102F7000091F08600120FFF78DF8681CC5B2082DF5
:102F8000E6DB70BD2DE9F04105460E461746984632
:102F9000FFF700FF10B90120BDE8F0816906080EB7
:102FA000FFF7C1FFFFF748FF18B9FFF723FF012024
:102FB000F2E73046FFF7B7FFFFF73EFF00240BE0D4
:102FC00018F80400FFF7AFFFFFF736FF18B9FFF757
:102FD00011FF0020E0E7641CBC42F1DBFFF70AFFB1
:102FE0000020D9E770B5054600246048001D006840
:102FF00020F470405D49091D08600846006840F4EF
:1030000000400860002617E000205949091F0860A9
:103010000220FFF73FF801205649C1F8A8016006D9
:10302000040E53488038006808B1601CC4B2022006
:10303000FFF730F8701CC6B2082EE5DB15B1FFF7BC
:103040002BFF01E0FFF74CFF204670BD2DE9F0415A
:1030500006460F4614461D46FFF79CFE10B9012098
:10306000BDE8F0817106080EFFF75DFFFFF7E4FE93
:1030700018B9FFF7BFFE0120F2E73846FFF753FF0C
:10308000FFF7DAFEFFF786FE012101EB4601C8B229
:10309000FFF749FFFFF7D0FE0DE0012C04D100201F
:1030A000FFF7A0FF287003E00120FFF79BFF2870C7
:1030B0006D1C601EC4B2002CEFD1FFF79BFE0020F8
:1030C000CEE770B505460E460024FFF763FE28469E
:1030D000FFF729FF641CFFF7AFFE3046FFF723FF21
:1030E000641CFFF7A9FEFFF755FE691CC8B2FFF785
:1030F0001AFF641CFFF7A0FE0020FFF773FF0446D1
:10310000FFF778FE204670BD2DE9F041074688465E
:1031100015461E460024FFF73DFE3846FFF703FF25
:10312000FFF78AFE4046FFF7FEFEFFF785FEFFF73A
:1031300031FE791CC8B2FFF7F6FEFFF77DFE00BF37
:103140000DE0681EA04204D00120FFF74BFF305570
:1031500003E00020FFF746FF3055601CC4B2AC42CC
:10316000EFDBFFF747FE2046BDE8F081000C014091
:10317000AC812142008021422DE9F04180460D467C
:1031800016461F460024FFF705FE4046FFF7CBFE1C
:10319000FFF752FE2846FFF7C6FEFFF74DFE00BFC1
:1031A00006E0385DFFF7BFFEFFF746FE601CC4B2C5
:1031B000B442F6DBFFF71EFE0120BDE8F08170B5DA
:1031C00005460E46144631462846FFF77AFF207022
:1031D000012070BD37B504460D4602AB01222946D9
:1031E0002046FFF7C9FF3EBD2DE9F8430746884654
:1031F00014461D46089E6A4641463846FFF7DFFFE3
:1032000028B3601CFF2101FA00F0C4F10801294431
:10321000491EFF220A41104300F0FF09C5F10800D2
:1032200006FA00F0C6B2C4F1070006419DF800009E
:1032300000EA090000909DF80000304300909DF8DE
:10324000002041463846FFF7C5FFBDE8F88300205F
:10325000FBE7F8B506460F4614461D466A46394652
:103260003046FFF7ACFF2DB10120A0409DF80010C3
:10327000084305E00120A0409DF8001021EA00006D
:10328000C0B200909DF8002039463046FFF7A2FFFB
:10329000F8BD0000014691F90020002A01DD002060
:1032A0001EE091F90020002A01DA042018E091F9CB
:1032B0000120002A01DD012012E091F90120002AFD
:1032C00001DA05200CE091F90220002A01DD02203C
:1032D00006E091F90220002A01DA062000E007202A
:1032E000704770B505462846FFF7D4FF0446E81C32
:1032F000FFF7D0FF44EAC00084B2A81DFFF7CAFF61
:1033000044EA801084B2204670BD70B588B0F3A145
:10331000F748FFF7DFFB02A905A801F0A6FF044666
:10332000072C41D101A801F011FA059804F0DCFB4B
:103330000646019904F038FC054604F099FB059017
:10334000069804F0D1FB0646019904F02DFC0546D1
:1033500004F08EFB0690079804F0C6FB0646019920
:1033600004F022FC054604F083FB079005A802F058
:10337000B6FA684601F007FABDF800100298484313
:103380000290BDF80010039848430390BDF8001068
:1033900004984843049002A802F034FB2246D5A1C9
:1033A000D348FFF797FB04E02246DBA1D048FFF7A4
:1033B00091FB08B070BD2DE9F04304460D46DDE9F0
:1033C00007670021012041E0DFF858C33CF8108076
:1033D000A0F1010CDFF84C9329F81C8009F1160CC0
:1033E0003CF81090A0F1010CDFF8388308F11608C2
:1033F00028F81C9008F1160C3CF81090A0F1010C74
:1034000008F1160828F81C9008F1160C3CF81090EA
:10341000A0F1010C08F1160828F81C9008F1160C10
:103420003CF81090A0F1010C08F1160828F81C9047
:1034300008F1160C3CF81090A0F1010C08F11608E8
:1034400028F81C9000F1010C0CF0FF000A28BBDBEF
:10345000DFF8D0C2ACF81240ACF82850ACF83E20EF
:10346000ACF85430ACF86A60ACF8807000210020F1
:1034700008E0DFF8B0C23CF910C0614400F1010C73
:103480000CF0FF000A28F4DB4FF00A0C91FBFCFC67
:103490000FFA8CFCDFF88C82A8F814C00021002001
:1034A0000AE0DFF880C20CF1160C3CF910C0614450
:1034B00000F1010C0CF0FF000A28F2DB4FF00A0CBF
:1034C00091FBFCFC0FFA8CF8DFF858C2ACF82A80AC
:1034D000002100200AE0DFF84CC20CF12C0C3CF972
:1034E00010C0614400F1010C0CF0FF000A28F2DB6F
:1034F0004FF00A0C91FBFCFC0FFA8CF8DFF824C2A9
:10350000ACF84080002100200AE0DFF818C20CF17E
:10351000420C3CF910C0614400F1010C0CF0FF00BA
:103520000A28F2DB4FF00A0C91FBFCFC0FFA8CF836
:10353000DFF8F0C1ACF85680002100200AE0DFF887
:10354000E4C10CF1580C3CF910C0614400F1010CCD
:103550000CF0FF000A28F2DB4FF00A0C91FBFCFC98
:103560000FFA8CF8DFF8BCC1ACF86C8000210020A9
:103570000AE0DFF8B0C10CF16E0C3CF910C06144F8
:1035800000F1010C0CF0FF000A28F2DB4FF00A0CEE
:1035900091FBFCFC0FFA8CF8DFF888C1ACF8828054
:1035A000BDE8F08338B50446032302226B21D02006
:1035B0000094FFF719FE38BD38B5044602230422F3
:1035C0001B21D0200094FFF70FFE38BD38B504460C
:1035D000022304221C21D0200094FFF705FE38BDF1
:1035E00010B50446234606226B21D020FFF731FE9A
:1035F00010BD10B54C4B01227521D020FFF784FD82
:103600004948007810BD10B5FFF7F3FF682801D1D5
:10361000012010BD0020FCE710B50446234605221A
:103620006A21D020FFF715FE10BD10B504462346D1
:1036300001223721D020FFF70CFE10BD10B502206B
:10364000FFF7B0FF0320FFF7B7FF0020FFF7BEFF33
:103650000020FFF7C5FF0020FFF7DEFF0020FFF787
:10366000E4FF10BD38B5002000906B4601227521A3
:103670006820FFF7EBFC9DF80000682806D09DF855
:1036800000202AA11A48FFF725FA05E09DF800203E
:1036900026A11748FFF71EFA00F065FDE0B9782073
:1036A00000F0C9F9782000F0ADFBC82000F08BFCD9
:1036B00002F07AF82148FFF714FE044602F07EF883
:1036C00040F2731002F0BBFCC82002F031FAFFF7A1
:1036D0001CFE012001F080FD38BD000072756E5F98
:1036E00073656C665F746573742E2E0D0A0000009E
:1036F0000044004073657474696E67206269617389
:103700002073756363657366756C6C79202E2E2E3D
:103710002564200D0A0000004661696C2E2E2025CC
:10372000640D0A00260100201801002077686F2030
:10373000616D20692025640D0A000000DC00002076
:103740002DE9F04F8DB00AA84E490BAB06AACDE982
:1037500000104D494D4802F0D1FD4A48008800F460
:10376000807000287ED0069804F0BEF904464FF021
:103770009D4104F087F846490860079804F0B4F9C1
:1037800004464FF09D4104F07DF8424908600898D6
:1037900004F0AAF904464FF09D4104F073F83E4945
:1037A0000860099804F0A0F904464FF09D4104F028
:1037B00069F83A490860384801684FF0804004F0E1
:1037C000F3F9019034480168019804F0EDF982465C
:1037D000304801684FF0404004F0E6F901902D4870
:1037E0000168019804F0E0F98346514604F0E4FAD8
:1037F00081464FF07E5103F0D7FF044603F0A8FF47
:10380000CDE90201224801684FF0804004F0CCF974
:10381000834620480168584604F0C6F981461E4890
:1038200001684FF0804004F0BFF983461B480168EF
:10383000584604F0B9F98246494603F0B5FF0446FC
:1038400003F086FF0746DDE9022303F093FA4FF009
:103850006632134BCDE9040103F086FD054603F003
:1038600049FB00E00BE00F4908600846006804F0DF
:10387000FFF8044622460CA10F48FFF72BF90DB0C4
:10388000BDE8F08FC0000020BA000020B400002086
:10389000CC000020D0000020D4000020D800002060
:1038A00066A64C40C80000205069746368203D2023
:1038B00025640D0A000000000044004038B50446AD
:1038C000FB4890F82400C0B114B10220009001E040
:1038D00000200090F64A1268D17BF54A52681078B1
:1038E0006B460122FFF74EFB10B14FF0FF3038BDA1
:1038F0009DF80010EE48417423E0ED48807A10B93D
:103900004FF0FF30F3E724B1E948407C08B10020D4
:10391000EDE714B10120009001E000200090E44A9E
:103920001268D17BE24A526810786B460122FFF799
:1039300029FB10B14FF0FF30D9E79DF80010DC48AB
:1039400041740020D3E738B5002419E0D848006856
:10395000C07AA04204D0D6480068407DA04200D181
:103960000CE0D349496808786B4601222146FFF7ED
:103970006DFB10B14FF0FF3038BD00BF601CC4B20A
:10398000CB4840680079A042E0DC0020F4E770B545
:1039900004460D46C6480068C07AA04204D0C44818
:1039A0000068407DA04202D14FF0FF3070BDC0489A
:1039B00040680079A04202DC4FF0FF30F6E7BC49D6
:1039C000496808782B4601222146FFF73FFBEDE7C7
:1039D00038B50446B64890F82300A04201D1002033
:1039E00038BD14B13020009001E000200090B048B4
:1039F000807C20B19DF8000040F002000090AC48AF
:103A000090F8220020B19DF8000040F08000009066
:103A1000A74A1268117DA64A526810786B460122A7
:103A2000FFF7B0FA10B14FF0FF30D9E7A04880F8A7
:103A300023400020D4E738B5044604F0700010B1EC
:103A40000120009005E014B10020009001E040202A
:103A50000090974A1268917C954A526810786B469C
:103A60000122FFF78FFA20B1002191488172481E90
:103A700038BD9DF8000020F040018D480173002002
:103A8000009004F0400020B99DF8000040F00400D0
:103A9000009004F0200020B99DF8000040F00200E2
:103AA000009004F0100020B99DF8000040F00100E3
:103AB000009004F0080020B99DF8000040F03800A4
:103AC00000907B4A1268D17C794A526810786B4624
:103AD0000122FFF757FA20B1002175488172481E74
:103AE000C6E724B1082C02D00020FFF771FF704810
:103AF0008472002101753220FEF7B0FA0020B7E78A
:103B000038B504466A48807CA04201D1002038BD07
:103B1000002C46D0664A12681179654A52681078BE
:103B20006B460122FFF792FA10B14FF0FF30EEE73B
:103B30009DF8000020F0200000905D4A1268117985
:103B40005B4A526810786B460122FFF71BFA10B1EE
:103B50004FF0FF30DBE70320FEF780FA02200090F1
:103B6000534890F8220020B19DF8000040F08000FA
:103B700000904F4890F8230020B19DF8000040F0DD
:103B8000300000904A4A1268117D494A5268107804
:103B90006B460122FFF7F6F9002851D04FF0FF30B5
:103BA000B5E7434A12681179414A526810786B466A
:103BB0000122FFF74BFA10B14FF0FF30A7E73C4866
:103BC000807A00F0010028B19DF8000040F020004C
:103BD000009004E09DF8000020F020000090344A9E
:103BE00012681179324A526810786B460122FFF749
:103BF000C9F910B14FF0FF3089E70320FEF72EFA24
:103C00002B4890F8220010B18020009001E00020A5
:103C10000090274890F8230020B19DF8000040F064
:103C200030000090224A1268117D214A52681078B3
:103C30006B460122FFF7A6F910B14FF0FF3066E79F
:103C40001B488474002062E708B51948807A10B9CF
:103C50004FF0FF3008BD00200090154A1268D17B5C
:103C6000134A526810786B460122FFF78BF910B1A6
:103C70004FF0FF30EEE70E4A126851790C4A526855
:103C800010786B460122FFF77DF910B14FF0FF303D
:103C9000E0E7074A12681179054A526810786B46C6
:103CA0000122FFF76FF928B14FF0FF30D2E7000093
:103CB000EC000020F74890F82400002850D00C2099
:103CC0000090F44A12681179F24A526810786B46F3
:103CD0000122FFF757F910B14FF0FF30BAE7C020CB
:103CE0000090EC48807A00F0010020B19DF80000BF
:103CF00040F020000090E74A12681179E54A5268C6
:103D000010786B460122FFF73DF910B14FF0FF30FC
:103D1000A0E7E048407C10B10220009001E00020C4
:103D20000090DC4A1268D17BDA4A526810786B4600
:103D30000122FFF727F910B14FF0FF308AE700208A
:103D40000090D44A12685179D24A526810786B4672
:103D50000122FFF717F9002852D04FF0FF3079E722
:103D600004200090CB4A12681179CA4A5268107830
:103D70006B460122FFF706F910B14FF0FF3069E7FB
:103D8000C448807C20B9C348807A00F0010010B993
:103D90004020009001E060200090BE4A1268117936
:103DA000BC4A526810786B460122FFF7EBF810B15D
:103DB0004FF0FF304EE7B748407C10B10120009033
:103DC00001E000200090B34A1268D17BB14A5268EA
:103DD00010786B460122FFF7D5F810B14FF0FF3095
:103DE00038E7AC4A12685179AA4A52681078A94B50
:103DF00010330122FFF7C6F810B14FF0FF3029E76A
:103E0000002027E770B50446002624F00104A148ED
:103E100090F8240008B1002070BD9E48807A10B947
:103E20004FF0FF30F8E79B48057C807A20409949A5
:103E300008740846007CA04202D04FF0FF3600E034
:103E4000002614B99348007D18B10120FFF736FD14
:103E500002E00020FFF732FD3CB1FFF7F5FE20B194
:103E60008C4805744FF0FF30D6E73046D4E738B5BC
:103E700004468848807A10B94FF0FF3038BDBC2C1A
:103E800002DB0120009015E0622C02DB0220009092
:103E900010E02A2C02DB032000900BE0142C02DB44
:103EA0000420009006E00A2C02DB0520009001E0CF
:103EB000062000907748C07A9DF80010884201D112
:103EC0000020DBE7734A12689178724A52681078D2
:103ED0006B460122FFF756F810B14FF0FF30CDE7E7
:103EE0009DF800106B48C1720020C7E738B5044642
:103EF000282C02DD4FF0FF3038BDDCB90020FFF781
:103F000067FD00208DF8000007208DF80100614A50
:103F10001268917C5F4A526810786B460222FFF764
:103F200031F810B14FF0FF30E6E700215948017534
:103F30000020E1E70120FFF74BFD20208DF8000075
:103F4000012C06D100208DF801000520FFF78FFF1E
:103F500017E0052C06DC01208DF801000520FFF795
:103F600086FF0EE0142C06DC02208DF801000A20EA
:103F7000FFF77DFF05E003208DF801001420FFF717
:103F800076FF9DF80100072101EB8010C0B28DF88B
:103F90000100404A1268917C3E4A526810786B4694
:103FA0000222FEF7EFFF10B14FF0FF30A4E7082127
:103FB0003848817200210173012101750020FFF74B
:103FC00021FF002098E738B504463248807A10B9BE
:103FD0004FF0FF3038BD2F4890F8240010B14FF05B
:103FE000FF30F7E72B48007D50B134B1282C04DCBA
:103FF000E0B2FFF77BFF0020ECE70020FFF776FF41
:10400000042C01DA042404E0B4F57A7F01DD4FF4D6
:104010007A744FF47A7090FBF4F0401EC0B20090B6
:104020001C4A126851781B4A526810786B4601226C
:10403000FEF7A8FF10B14FF0FF30CBE79DF800006E
:10404000401C4FF47A7191FBF0F081B21148C181AC
:104050000146C9894810FFF70AFF0020BAE738B5C2
:1040600004460C48807A10B94FF0FF3038BD022C5E
:1040700006D0042C07D0082C08D0102C0FD10BE050
:10408000002000900EE0082000900BE0102000902F
:1040900008E00000EC0000201820009002E04FF043
:1040A000FF30E3E700BFF948407A9DF80010B0EB1D
:1040B000E10F01D10020D9E7F44A1268D179F34A1F
:1040C000526810786B460122FEF75CFF10B14FF08A
:1040D000FF30CBE79DF80000C110EC484172002092
:1040E000C4E738B50446E948807A10B94FF0FF308C
:1040F00038BDFA2C09D0B4F5FA7F09D0B4F57A7F2F
:1041000009D0B4F5FA6F0CD108E0002000900BE064
:104110000820009008E01020009005E01820009092
:1041200002E04FF0FF30E3E700BFD848007A9DF887
:104130000010B0EBE10F01D10020D9E7D34A12689B
:104140009179D24A526810786B460122FEF71AFF25
:1041500010B14FF0FF30CBE79DF80000C010CB4905
:1041600008720020C4E71CB580208DF80000C74A03
:104170001268917CC54A526810786B460122FEF79E
:1041800001FF10B14FF0FF301CBD6420FDF766FF4A
:1041900000208DF80000BD4A1268917CBB4A52682D
:1041A00010786B460122FEF7EDFE10B14FF0FF30A4
:1041B000EAE7B64A1268917DB44A526810786B46B5
:1041C0000622FEF743FF10B14FF0FF30DCE79DF809
:1041D0000500C007400F9DF8031001F0010140EAFF
:1041E00041009DF8011001F0010140EA010494B181
:1041F000012C03D10121A548C17431E0022C03D167
:104200000021A248C1742BE02146A1A002F0FEF9D2
:104210004FF0FF30B8E79D4A1268D1789B4A526848
:1042200010786B460122FEF711FF10B14FF0FF30FE
:10423000AAE79DF8000000F00F042CB99E4802F098
:10424000E5F94FF0FF309FE7042C06D19BA002F068
:10425000DDF901218D48C17402E000218B48C17451
:10426000FF218A488172FF2088490872FF21874810
:104270004172C1724FF6FF71C181FF2101748174D7
:104280000121017380F82210002180F8231041756C
:1042900001751630016041608160163880F8241085
:1042A00080F82510C1844FF4FA60FFF71AFF10B1AF
:1042B0004FF0FF3068E70220FFF7D1FE10B14FF05A
:1042C000FF3061E72A20FFF7D2FD10B14FF0FF3039
:1042D0005AE73220FFF777FE10B14FF0FF3053E777
:1042E0000020FFF78FFD10B14FF0FF304CE70020AA
:1042F000FFF706FC10B14FF0FF3045E70020FFF755
:104300009AFB002040E770477CB504460D465F48A5
:10431000807A00F0700010B94FF0FF307CBD5B4A2E
:104320001268117B594A526810786B460622FEF7D4
:104330008DFE10B14FF0FF30F0E79DF801009DF8C1
:10434000001040EA012000B220809DF803009DF893
:10435000021040EA012000B260809DF805009DF83F
:10436000041040EA012000B2A08015B12846FFF7F2
:10437000CAFF0020D2E77CB504460D464348807A48
:1043800000F0080010B94FF0FF307CBD3F4A1268C2
:10439000517B3E4A526810786B460622FEF756FE65
:1043A00010B14FF0FF30F0E79DF801009DF80010CC
:1043B00040EA012000B220809DF803009DF8021021
:1043C00040EA012000B260809DF805009DF80410CD
:1043D00040EA012000B2A08015B12846FFF793FF04
:1043E0000020D2E72DE9FE4F05460C462748807A8B
:1043F00018B94FF0FF30BDE8FE8F244A1268917B58
:10440000224A5268107802AB0222FEF71FFE10B15A
:104410004FF0FF30EFE79DF809009DF8081040EAE3
:10442000012006B214B12046FFF76DFF1749496815
:10443000C88803F071FB154901904968B1F908007B
:1044400003F052FB8346304603F04EFB5946009082
:1044500003F0B2FC8246019903F014FA81461F4929
:1044600003F0A2F980464FF08F4103F09DFB074611
:1044700003F0FEFA28600020BDE710B588B00446BE
:104480001CB94FF0FF3008B010BD29E0EC0000204F
:10449000556E737570706F7274656420736F667497
:1044A000776172652070726F6475637420726576CF
:1044B0002025642E0A000000808C000848616C668C
:1044C0002073656E7369746976697479207061729E
:1044D0007420666F756E642E0D0A000000000C4299
:1044E000206830B9606820B9A06810B9002008B011
:1044F00010BDFA494968087806AB03221146FEF759
:10450000A5FD10B14FF0FF30F1E79DF8180008212C
:1045100001EB201000F00F00ADF800009DF819002D
:1045200001EB201000F00F00ADF802009DF81A001A
:1045300001EB201000F00F00ADF8040020684100EE
:10454000BDF90000403091FBF0F000B2ADF8100072
:1045500060684100BDF90200403091FBF0F000B20C
:10456000ADF81200A0684100BDF90400403091FB95
:10457000F0F000B2ADF81400D8494968087806ABED
:1045800006221146FEF762FD10B14FF0FF30AEE794
:104590009DF819009DF8181040EA012000B2ADF80E
:1045A00008009DF81B009DF81A1040EA012000B297
:1045B000ADF80A009DF81D009DF81C1040EA01208E
:1045C00000B2ADF80C00BDF81000BDF808100844AA
:1045D00000B2ADF81000BDF81200BDF80A10084492
:1045E00000B2ADF81200BDF81400BDF80C1008447C
:1045F00000B2ADF81400BDF81000000A8DF81800E4
:10460000BDF81000C0B28DF81900BDF81200000A04
:104610008DF81A00BDF81200C0B28DF81B00BDF86D
:104620001400000A8DF81C00BDF81400C0B28DF80B
:104630001D00AA494968087806AB06221146FEF714
:10464000A1FC10B14FF0FF3051E700204FE70146C9
:10465000A248007A30B1012807D0022809D00328E7
:104660000FD10AE0FA2008800EE04FF4FA700880BB
:104670000AE04FF47A70088006E04FF4FA60088090
:1046800002E00020088000BF00BF00207047014604
:104690009248407A30B1012807D0022808D0032878
:1046A0000CD108E0022008700BE00420087008E03C
:1046B0000820087005E01020087002E04FF0FF307D
:1046C000704700BF8548C07C18B108784006000ECE
:1046D00008700020F4E701468048C07A082817D205
:1046E000DFE800F01704070A0D101318BC2008803B
:1046F00013E06220088010E02A2008800DE01420DA
:1047000008800AE00A20088007E00520088004E00D
:1047100000BF00BF0020088000BF00BF002070471E
:1047200001466E4890F8240010B14FF0FF307047FA
:104730006A48C08908800020F9E701460020088007
:10474000401E704701464FF0FF30704701466348F6
:10475000007A30B1012807D0022808D003280CD1F4
:1047600008E05F4808600BE05E48086008E05E48CB
:10477000086005E05D48086002E04FF0FF307047D8
:1047800000BF0020FBE701465448407A30B10128C1
:1047900008D002280AD0032810D10BE04FF4804043
:1047A00008800EE041F69C7008800AE04FF48050CB
:1047B000088006E04FF40060088002E04FF0FF3010
:1047C000704700BF4548C07C10B108884010088081
:1047D0000020F5E701464148007C08700020704742
:1047E00001463E48807A10B10120087001E00020A7
:1047F00008700020704738B504463848807A10B9F0
:104800004FF0FF3038BD354A1268117C334A526888
:1048100010786B460222FEF719FC10B14FF0FF3002
:10482000F0E79DF801009DF8001040EA012000B279
:1048300020800020E6E72DE9FE4F07468846924695
:104840001D46DDF830B000260024244890F82400EE
:1048500010B1601EBDE8FE8F002028701F48807ACE
:1048600010B94FF0FF30F5E71C48007C10B94FF04D
:10487000FF30EFE71948007C00F0400008B1B01CA1
:10488000C6B21648007C00F0200008B1B01CC6B2C9
:104890001248007C00F0100008B1B01CC6B20F48EE
:1048A000007C00F0080008B1B01DC6B20B4A1268C7
:1048B000917A0A4A526810786B460222FEF7C6FBCC
:1048C00010B14FF0FF30C5E79DF801009DF80010D2
:1048D00040EA0129B1450BDA0020BBE7EC000020DB
:1048E00000000343000083423333034233338341E8
:1048F000FC4840684088B9EB600F17DDF94A126840
:10490000517CF84A526810786B460122FEF79EFBF4
:1049100010B14FF0FF309DE79DF8000000F010004F
:1049200020B1FFF791F96FF0010093E75046FFF7D0
:10493000EAFCEC4A1268D17AEA4A526810786B466F
:104940003246FEF783FB10B14FF0FF3082E799FB50
:10495000F6F0401E8BF8000000202870B4422AD0E8
:10496000E048007C00F0080028B3601C1DF800003F
:104970001DF8041040EA012000B2A8F80000E01C75
:104980001DF80010A01C1DF8000041EA002000B234
:10499000A8F80200601D1DF80010201D1DF8000081
:1049A00041EA002000B2A8F80400287840F008008E
:1049B0002870A01D84B2B44213D0CA48007C00F015
:1049C000400070B1601C1DF800001DF8041040EAA2
:1049D000012000B23880287840F040002870A01CE8
:1049E00084B2B44213D0BF48007C00F0200070B104
:1049F000601C1DF800001DF8041040EA012000B200
:104A00007880287840F020002870A01C84B2B4423E
:104A100013D0B448007C00F0100070B1601C1DF889
:104A200000001DF8041040EA012000B2B880287888
:104A300040F010002870A01C84B200200AE7F8B5EE
:104A400004460F461646A74890F8240010B94FF0C8
:104A5000FF30F8BDA348807A10B94FF0FF30F8E777
:104A6000A04A1268917A9F4A526810786B460222D7
:104A7000FEF7ECFA10B14FF0FF30EAE79DF80100C5
:104A80009DF8001040EA0125A54203DA00203070AD
:104A9000401EDEE7934840684088B5EB600F17DDA5
:104AA000904A1268517C8F4A526810786B460122F6
:104AB000FEF7CCFA10B14FF0FF30CAE79DF80000C6
:104AC00000F0100020B1FFF7BFF86FF00100C0E761
:104AD000E2B2844B1B68D97A824B5B6818783B46FC
:104AE000FEF7B4FA10B14FF0FF30B2E795FBF4F0E7
:104AF000401E30700020ACE701467A4880F8221052
:104B0000002070477CB5054676494968087801ABB6
:104B100004220D21FEF79AFA08B107207CBD9DF80A
:104B20000700C0F301109DF8041001F0E00140EA15
:104B3000E1008DF800009DF80700C0F381009DF8AA
:104B4000051001F0E00140EAE1008DF801009DF858
:104B5000070000F003009DF8061001F0E00140EAB4
:104B6000E1008DF8020000241CE01DF8040018B9D3
:104B7000002045F8240013E05B4845F8240006E0D7
:104B800055F82400594903F00FF845F824001DF8A2
:104B90000400401EC0B20DF804000028F0D100BF90
:104BA000601CC4B2032CE0DB0020B7E72DE9FE4F08
:104BB00006460F4600256846FFF7A4FF002442E0A2
:104BC00056F8240057F82410A0EB010ABAF1000FA0
:104BD00001DB514601E0CAF10001084602F084FF02
:104BE00083464FF08F4102F04DFE80465DF8240071
:104BF000002102F009FF16D05DF82410404602F0B3
:104C000041FE82464FF07E5103F0D6F8814629F0EE
:104C1000004A3748416A504603F092F812D2012008
:104C2000A04005430EE03248C169404602F088FFCB
:104C300005D32F48016A404603F082F802D20120D2
:104C4000A0400543641C032CBADB2846BDE8FE8F58
:104C50002DE9FC5F06460F46002522494968087881
:104C600001AB03220D21FEF7F1F910B10720BDE8D9
:104C7000FC9F9DF8040000F01F008DF804009DF8D3
:104C8000050000F01F008DF805009DF8060000F0FB
:104C90001F008DF80600002462E056F8240057F843
:104CA0002410A0EB010BBBF1000F01DB594601E022
:104CB000CBF10001084602F017FF4FF08F41009042
:104CC00002F0E0FD814601A8005DC0B30849086814
:104CD00002F022FF83465946064802F0D3FD804683
:104CE0000FE00000EC0000207B14AE3E1D5A843F14
:104CF000BC7F000800B04C45FE49404602F054FF1E
:104D0000804601A8005D401EC0B201A908550028D8
:104D1000F2D14146484602F0B5FD83464FF07E5140
:104D200003F04AF882462AF0004BF348816958465E
:104D300003F006F813D20120A04005430FE0FFE77F
:104D4000ED480169484602F0FBFE05D3EA48416997
:104D5000484602F0F5FF02D20120A0400543641C42
:104D6000032C9ADB284682E72DE9F04F87B00546F1
:104D70000C46914601208DF8100000208DF811009E
:104D8000DE4A1268917CDD4A5268107804AB022238
:104D9000FEF7F8F820B14FF0FF3007B0BDE8F08F14
:104DA000C820FDF75BF900208DF81000D34A126887
:104DB000D17BD24A5268107804AB0122FEF7E2F8A8
:104DC00010B14FF0FF30E8E7CC4A12685179CB4A76
:104DD0005268107804AB0122FEF7D4F810B14FF0FE
:104DE000FF30DAE7C54A1268917CC44A52681078ED
:104DF00004AB0122FEF7C6F810B14FF0FF30CCE74C
:104E0000BE4A1268D17DBD4A5268107804AB0122B7
:104E1000FEF7B8F810B14FF0FF30BEE7B74A12689E
:104E20001179B64A5268107804AB0122FEF7AAF84D
:104E300010B14FF0FF30B0E70C208DF81000AF4AF2
:104E400012681179AD4A5268107804AB0122FEF75E
:104E500099F810B14FF0FF309FE70F20FDF7FEF8F3
:104E6000A648806A407A8DF81000A44A12689178AA
:104E7000A24A5268107804AB0122FEF783F810B101
:104E80004FF0FF3089E79D48806A007A8DF8100066
:104E90009A4A12685178994A5268107804AB0122F4
:104EA000FEF770F810B14FF0FF3076E7B9F1000F60
:104EB00007D09248806A807A40F0E0008DF81000B8
:104EC00004E08E48806A807A8DF810008B4A126860
:104ED00091798A4A5268107804AB0122FEF752F8A1
:104EE00010B14FF0FF3058E7B9F1000F07D08348F9
:104EF000806AC07A40F0E0008DF8100003E07E4840
:104F0000C07A8DF810007D4A1268D1797B4A5268C8
:104F1000107804AB0122FEF735F810B14FF0FF30E6
:104F20003BE7B9F1000F02D0C820FDF797F8402009
:104F30008DF81000714A12681179704A5268107821
:104F400004AB0122FEF71EF810B14FF0FF3024E74A
:104F500078208DF81000694A12685179674A5268C2
:104F6000107804AB0122FEF70DF810B14FF0FF30BE
:104F700013E761498889FDF771F800208DF810006A
:104F80005E4A126851795D4A5268107804AB01227A
:104F9000FDF7F8FF10B14FF0FF30FEE6574A1268F8
:104FA000917A564A5268107804AB0222FEF74EF806
:104FB00010B14FF0FF30F0E69DF811009DF8101091
:104FC00040EA012B0C209BFBF0F0C6B20020A86049
:104FD00068602860A06060602060824665E0474AA3
:104FE0001268D17A454A5268107804AB0C22FEF759
:104FF0002DF810B14FF0FF30CFE69DF811009DF86D
:10500000101040EA012000B2ADF808009DF813002E
:105010009DF8121040EA012000B2ADF80A009DF898
:1050200015009DF8141040EA012000B2ADF80C0004
:10503000BDF90810206808442060BDF90A106068B6
:1050400008446060BDF90C10A0680844A0609DF899
:1050500017009DF8161040EA012000B2ADF80000DC
:105060009DF819009DF8181040EA012000B2ADF833
:1050700002009DF81B009DF81A1040EA012000B2C2
:10508000ADF80400BDF90010286808442860BDF997
:105090000210686808446860BDF90410A8680844F4
:1050A000A8600AF1010000F0FF0AB24597DB124840
:1050B000D0F800C02868C117090441EA104107046C
:1050C00062460023384601F07CFA32460023CDE9DF
:1050D000020101F076FA28600748D0F800C068683D
:1050E000C117090441EA104107046246002338460B
:1050F00006E0000054E3853FBC7F0008EC00002080
:1051000001F05FFA32460023CDE9020101F059FABD
:105110006860F948D0F800C0A868C117090441EADE
:105120001041070462460023384601F04AFA32462D
:105130000023CDE9020101F044FAA860EE48D0F85E
:1051400004C02168C817000440EA11480F046246F1
:1051500000233846414601F034FA32460023CDE9B7
:10516000020101F02EFA2060E348D0F804C0606824
:10517000C117090441EA104107046246002338467A
:1051800001F01FFA32460023CDE9020101F019FABD
:105190006060D948D0F804C0A068C117090441EA8A
:1051A0001041070462460023384601F00AFA3246ED
:1051B0000023CDE9020101F004FAA060A0680028F4
:1051C00004DDA068A0F58030A06003E0A06800F5D1
:1051D0008030A0600020E0E538B50446C74890F86C
:1051E0002400A04201D1002038BD44B3C34890F848
:1051F000250010B94FF0FF30F6E70020FEF75EFB08
:105200000020FEF77DFCBD49C88CFEF7DCFE0020C7
:105210000090BA49496808786B4601222321FDF7BE
:10522000B1FE0121B54880F824100120FEF746FBAD
:10523000FEF70AFDB2A1B948FDF74CFC13E00020CF
:10524000FEF73CFBAD48007C0090AC49496808780B
:105250006B4601222321FDF795FE0021A74880F827
:105260002410FEF7F1FC0020BEE72DE9F04F8DB0D1
:1052700083460F4602200C90A04890F8240020B1ED
:105280000020FFF7A9FF012600E0002603A8FFF792
:10529000DEF905A8FFF7FBF901A8FFF71CFA02A841
:1052A000FFF73EFA954890F80AA004A8FFF792FA93
:1052B000002407E0002239465846FFF755FD00B9A3
:1052C00002E0641C022CF5DB00BF022C01D100259A
:1052D00028E0002407E0012206A909A8FFF744FD01
:1052E00000B902E0641C022CF5DB00BF022C01D1E6
:1052F000002517E006A93846FFF758FC00F0FF0824
:1053000009A95846FFF7A4FC00F0FF090025B9F1F0
:10531000000F01D145F00105B8F1000F01D145F0B2
:10532000020500BFFF2075490872FF2173484172D2
:10533000C1724FF6FF71C181FF2181720174012199
:105340000173BDF80C00FEF7CCFE9DF81400FEF7CB
:1053500086FEBDF80400FEF78AFDBDF80800FEF7E2
:1053600032FE5046FEF767FB9DF81000FEF74AFD3F
:105370003EB10120FFF730FF2A4669A16748FDF7DB
:10538000A9FB2A4669A16548FDF7A4FB28460DB094
:10539000BDE8F08FF8B504460D46164616B94FF035
:1053A000FF30F8BD5548807A10B94FF0FF30F8E76C
:1053B00020128DF80000E0B28DF801009DF8010088
:1053C00028444E4949684989884202DD4FF0FF3040
:1053D000E7E74A4A1268117E484A526810786B46DD
:1053E0000222FDF7CFFD10B14FF0FF30D9E7EAB24E
:1053F000424B1B68597D414B5B6818783346FDF77B
:10540000C1FD10B14FF0FF30CBE70020C9E7F8B580
:1054100004460D46164616B94FF0FF30F8BD374822
:10542000807A10B94FF0FF30F8E720128DF80000B5
:10543000E0B28DF801009DF8010028442F49496829
:105440004989884202DD4FF0FF30E7E72B4A1268B6
:10545000117E2A4A526810786B460222FDF792FDAF
:1054600010B14FF0FF30D9E7EAB2244B1B68597DE9
:10547000224B5B6818783346FDF7E8FD10B14FF01A
:10548000FF30CBE70020C9E72DE9F04385B00546A2
:105490000E4690469946194890F8250020B14FF0E5
:1054A000FF3005B0BDE8F08316B94FF0FF30F8E7E4
:1054B000002447E0281B102801DD102000E0281BF5
:1054C00087B2321939462046FFF764FF10B14FF01A
:1054D000FF30E6E701AA39462046FFF798FF10B1F2
:1054E0004FF0FF30DDE730193A4601A901F00AF923
:1054F00030B36FF00100D4E7BC7F0008EC0000205F
:105500006D70755F7365745F646D705F73746174E3
:105510006520646D70206F6E0D0A0000004400402D
:10552000646D70206F6E0D0A000000007265747566
:10553000726E2E2E726573203D2025640D0A0000C8
:10554000E01984B2AC42B5DB4FEA28208DF80000A8
:1055500008F0FF008DF80100924A1268917E914A8E
:10556000526810786B460222FDF70CFD10B14FF027
:10557000FF3096E701218B4880F82510A0F826908F
:1055800000208EE70146874890F82400087000202C
:10559000704702464FF0FF30704701464FF0FF3032
:1055A0007047F8B505460F461446002C70D0B5F587
:1055B000FF5F01DDFF2605E0202D01DA012601E075
:1055C000C5F3471607B90127282C02DD4FF0FF303D
:1055D000F8BD7448407D28BB724890F8240038B16B
:1055E0000020FFF7F9FD01216E4880F8201003E04C
:1055F00000216C4880F820106A481630FFF727F821
:1056000068481830FFF743F866481A30FFF763F828
:1056100064481C30FFF784F86248817A81771F3034
:10562000FFF7D8F80020FEF749F90020FEF75EFCEE
:1056300000208DF800005B4A12689178594A526840
:1056400010786B460122FDF79DFC10B14FF0FF3042
:10565000BEE740208DF80000524A1268D17B514AC3
:10566000526810786B460122FDF78CFC00B165E0B2
:105670008DF800608DF801704A4A1268117A494A23
:10568000526810786B460222FDF77CFC08B155E0A9
:1056900047E00520FCF7E2FC4248407A072101EB95
:1056A000C000C0B28DF800003E4A1268D1793D4A70
:1056B000526810786B460122FDF764FC00B13DE0B2
:1056C00020208DF80000012C03D100208DF801006E
:1056D0000EE0052C03DC01208DF8010008E0142CFD
:1056E00003DC02208DF8010002E003208DF80100A8
:1056F0009DF80100072101EB8010C0B28DF8010078
:10570000284A1268917C274A526810786B46022218
:10571000FDF738FC00B111E001212248417500205D
:1057200056E7204A1632002103E0505C00B105E044
:10573000491C0C29F9D34FF0FF3049E7FF201949E4
:105740000872FF2117484172C1724FF6FF71C18183
:10575000FF2181720174012101730146887FFEF7E8
:105760006AF91049C88AFEF7BCFC0E49087EFEF7AC
:1057700076FC0C49488BFEF77AFB0A49888BFEF7CA
:1057800022FC0849C87FFEF73DFB064890F8200040
:1057900010B10120FFF720FD0021024841750020D3
:1057A00016E70000EC00002010B5C8234FF480621B
:1057B000F74940F6F630FFF767FE10BD10B586B02A
:1057C0000446F4A000680390F3A000680290F3A0E0
:1057D00000680190F2A00068009004F0030003A9A3
:1057E000085C8DF8140003A8C4F3C101405C8DF877
:1057F000150003A8C4F38111405C8DF8160004F075
:10580000030002A9085C8DF8100002A8C4F3C101CE
:10581000405C8DF8110002A8C4F38111405C8DF842
:10582000120005AA032140F22640FFF7B3FD18B18C
:105830004FF0FF3006B010BD04AA032140F22A4009
:10584000FFF7A8FD10B14FF0FF30F3E70198059086
:105850000098049004F0040058B19DF8140040F042
:1058600001008DF814009DF8100040F001008DF843
:10587000100004F0200058B19DF8150040F0010020
:105880008DF815009DF8110040F001008DF8110011
:1058900004F4807058B19DF8160040F001008DF8B6
:1058A00016009DF8120040F001008DF8120005AAC4
:1058B00003214FF48860FFF76DFD10B14FF0FF300A
:1058C000B8E704AA032140F23140FFF763FD10B1AD
:1058D0004FF0FF30AEE7B34804810020AAE71FB5C0
:1058E0000446B048007A00F0030054F8200001900C
:1058F000AC48007A00F0040010B1019840420190D9
:10590000A848007AC0F3C10054F820000290A548CE
:10591000007A00F0200010B1029840420290A148A5
:10592000007AC0F3811054F8200003909D4800894C
:1059300000F4807010B10398404203909A49019896
:1059400080FB0101800F40EA810001909649029896
:1059500080FB0110820042EA917002909249039804
:1059600080FB0110820042EA917003900198000EC2
:105970008DF800000198000C8DF801000198000AD4
:105980008DF802000198C0B28DF803006A46042128
:105990004FF47470FFF7FEFC18B14FF0FF3004B005
:1059A00010BD0298000E8DF800000298000C8DF8D2
:1059B00001000298000A8DF802000298C0B28DF82A
:1059C00003006A4604214FF47570FFF7E3FC10B141
:1059D0004FF0FF30E3E70398000E8DF800000398C6
:1059E000000C8DF801000398000A8DF8020003985E
:1059F000C0B28DF803006A4604214FF47670FFF7B9
:105A0000C9FCCCE770B588B0064601A8FEF7BBFE1E
:105A1000BDF804000021C90341EA5045C4036148B0
:105A2000007A00F0030056F8200005905D48007AE7
:105A300000F0040010B10598404205905948007AE2
:105A4000C0F3C10056F8200006905648007A00F0D6
:105A5000200010B10698404206905248007AC0F3E8
:105A6000811056F8200007904E48008900F480709D
:105A700010B10798404207900598C117A0FB042376
:105A800001FB043100FB0510810041EA9270059092
:105A90000698C117A0FB042301FB043100FB05108D
:105AA000810041EA927006900798C117A0FB042379
:105AB00001FB043100FB0510810041EA9270079060
:105AC0000598000E8DF808000598000C8DF8090067
:105AD0000598000A8DF80A000598C0B28DF80B00F1
:105AE0000698000E8DF80C000698000C8DF80D003D
:105AF0000698000A8DF80E000698C0B28DF80F00C7
:105B00000798000E8DF810000798000C8DF8110012
:105B10000798000A8DF812000798C0B28DF813009C
:105B200002AA0C214FF42570FFF734FC08B070BDB9
:105B300030B585B004461DA207CA02AB07C3C82C06
:105B400003DD4FF0FF3005B030BDC82090FBF4F00E
:105B5000401E85B2280A8DF80000E8B28DF80100D9
:105B60006A46022140F21620FFF714FC10B14FF0F4
:105B7000FF30E8E702AA0C2140F6C120FFF70AFC3B
:105B800010B14FF0FF30DEE7064884810020DAE7ED
:105B9000E47F00084CCD6C000CC92C003656760012
:105BA00026466600AC01002009E3CA02FEF2ABC43F
:105BB000AAF1DFDFBBAFDFDF0146FC488089088048
:105BC000002070472DE9FC4706460F4606F0070007
:105BD00010B1B7F5C86F03DD4FF0FF30BDE8FC87AB
:105BE000384601F099FF8146F14901F04BFE8046AD
:105BF0006846FEF74CFD9DF80000022806D00428F8
:105C000016D0082826D0102848D135E04FF08D4115
:105C1000404601F0C9FF814601F046FF84B2E549E4
:105C2000404601F0C1FF814601F03EFF85B238E0F9
:105C30004FF08C41404601F0B7FF814601F034FF40
:105C400084B2DD49404601F0AFFF814601F02CFFF0
:105C500085B226E04FF08B41404601F0A5FF81461A
:105C600001F022FF84B2D549404601F09DFF8146F4
:105C700001F01AFF85B214E04FF08A41404601F06E
:105C800093FF814601F010FF84B2CD49404601F0F8
:105C90008BFF814601F008FF85B202E04FF0FF3034
:105CA0009CE700BF20128DF80400E0B28DF80500DB
:105CB00028128DF80600E8B28DF8070006F0010002
:105CC000A0B101AA02214FF4EA70FFF763FB10B103
:105CD0004FF0FF3082E70DF1060202214FF492707F
:105CE000FFF758FB10B14FF0FF3077E706F00200E6
:105CF000A0B101AA02214FF4EC70FFF74BFB10B1E9
:105D00004FF0FF306AE70DF1060202214FF4947064
:105D1000FFF740FB10B14FF0FF305FE706F00400E3
:105D2000A0B101AA02214FF4EE70FFF733FB10B1CE
:105D30004FF0FF3052E70DF1060202214FF496704A
:105D4000FFF728FB10B14FF0FF3047E7002045E791
:105D500038B504460020009004F0010020B19DF801
:105D6000000040F03000009004F0020020B19DF8E7
:105D7000000040F00C00009004F0040020B19DF8F9
:105D8000000040F0030000906A4601214FF4A47027
:105D9000FFF700FB38BD38B50446012C01DA0124B9
:105DA00002E0042C00DD0424601EC0B200906A46AC
:105DB000012140F24F10FFF7EDFA38BD38B5044627
:105DC000052094FBF0F085B228128DF80000E8B2AF
:105DD0008DF801006A4602214FF4EF70FFF7DAFAFE
:105DE00038BD38B50446052094FBF0F085B2281282
:105DF0008DF80000E8B28DF801006A4602214FF4E8
:105E0000ED70FFF7C7FA38BDF8B505460E464FF4FA
:105E10007A7095FBF0F000FB06F4200E8DF8000080
:105E2000200C8DF80100200A8DF80200E0B28DF8F8
:105E300003006A4604214FF4AE70FFF7ABFAF8BDD9
:105E400038B50446052094FBF0F084B220128DF89A
:105E50000000E0B28DF801006A4602214FF4AD70F7
:105E6000FFF798FA38BD38B50446052094FBF0F0EA
:105E700084B220128DF80000E0B28DF801006A466D
:105E800002214FF4AC70FFF785FA38BD38B50446EF
:105E900014B94FF0FF3038BD6A4604214FF45870F2
:105EA000FFF7B5FA10B14FF0FF30F4E79DF80000AE
:105EB00000069DF8011040EA01409DF8021040EAFA
:105EC00001209DF80310084320600020E3E738B567
:105ED0000446200E8DF80000200C8DF80100200AE9
:105EE0008DF80200E0B28DF803006A4604214FF4F9
:105EF0005870FFF74FFA38BD38B5044614B94FF063
:105F0000FF3038BD6A4604214FF47170FFF77FFA05
:105F100010B14FF0FF30F4E79DF8000000069DF847
:105F2000011040EA01409DF8021040EA01209DF86E
:105F30000310084300EB8000800020600020E0E7B1
:105F400038B504461420B4FBF0F4200E8DF80000A0
:105F5000200C8DF80100200A8DF80200E0B28DF8C7
:105F600003006A4604214FF47170FFF713FA38BD3D
:105F700038B5044664B120208DF8000028208DF843
:105F8000010030208DF8020038208DF8030004E075
:105F9000A3220421684600F0E1FB6A46042140F692
:105FA0009E20FFF7F7F9FDF74FFE38BDAC0100204A
:105FB00000004843000040460000C0450000404546
:105FC0000000C04438B5044664B1C0208DF800001C
:105FD000C2208DF80100C4208DF80200C6208DF883
:105FE000030004E08B220421684600F0B7FB6A46F8
:105FF000042140F69820FFF7CDF9FDF725FE38BDC6
:106000003EB504466CB1FDA1D1E900208968CDE917
:10601000002002916A4609214FF49760FFF7BAF910
:106020003EBDF9A2D2E900109268CDE901020091CB
:106030006A4609214FF49760FFF7ACF9F0E73EB5E7
:10604000044602208DF80000CA208DF80100E320EC
:106050008DF8020009208DF803006A4604216820AB
:10606000FFF798F9A3208DF8000004F0400048B134
:10607000C0208DF80100C8208DF80200C2208DF8E4
:10608000030006E0A3208DF801008DF802008DF8D2
:10609000030004F4C07048B1C4208DF80400CC2083
:1060A0008DF80500C6208DF8060006E0A3208DF8C7
:1060B00004008DF805008DF80600A3208DF8070078
:1060C0008DF808008DF809006A460A2140F6A720DD
:1060D000FFF760F904F0030018B120208DF80000EC
:1060E00002E0D8208DF800006A46012140F6B62073
:1060F000FFF750F904F0200018B10120FFF780FFEE
:1061000002E00020FFF77CFF04F4C07008B304F441
:10611000807060B1B2208DF800008B208DF80100F6
:10612000B6208DF802009B208DF803000BE0B02014
:106130008DF8000080208DF80100B4208DF8020059
:1061400090208DF803006A46042140F6A220FFF754
:1061500021F904F0010020B3F8208DF800006A4610
:1061600001214FF40B60FFF715F9FA210720FFF723
:1061700029FD0720FFF7ECFD0120FFF70CFE64204E
:10618000FFF71CFE4FF4FA70FFF72BFEC821A14861
:10619000FFF73AFE2820FFF753FE0A20FFF763FEC1
:1061A00008E0D8208DF800006A4601214FF40B600A
:1061B000FFF7F0F804F0020018B1D9208DF80000C4
:1061C00002E0D8208DF800006A46012140F23D70BF
:1061D000FFF7E0F804F0040018B10120FFF7F2FE29
:1061E00002E00020FFF7EEFE04F0100018B10120DD
:1061F000FFF7BEFE02E00020FFF7BAFE44F0080001
:1062000085494881FDF720FD00208349887304F00B
:10621000400018B10846807B801D887304F4C0706C
:1062200020B17D48807B801D7B49887304F0140079
:1062300020B17948807B10307749887304F00300DF
:1062400020B17548807B001D7349887300203EBDD6
:106250000146714840890880002070472DE9F041CF
:106260000446E07800F0C006E07800F03F05607872
:1062700000F0010098B1EF102846E91705EB5171C5
:10628000C910A5EBC101491C01F0FF086248006874
:1062900020B16148414602683846904700BF6078A7
:1062A00000F0080030B15C48406818B1B0115A4A9B
:1062B000516888470020BDE8F08110B586B00446DB
:1062C00056A207CA03AB07C357A207CA8DE8070047
:1062D000012C09D0022C0ED103AA0B2140F68220FA
:1062E000FFF758F806B010BD6A460B2140F6822031
:1062F000FFF750F8F6E74FF0FF30F3E72DE9F04FE6
:106300008DB00746884615469946DDE9166B002490
:10631000002030804049887B5A4605A9FEF78FFB54
:1063200018B1601E0DB0BDE8F08F3B48807A00F0D8
:106330001400002861D09DF8140000069DF8151087
:1063400040EA01409DF8161040EA01209DF8171020
:10635000084328609DF8180000069DF8191040EACF
:1063600001409DF81A1040EA01209DF81B100843D7
:1063700068609DF81C0000069DF81D1040EA014071
:106380009DF81E1040EA01209DF81F100843A860E8
:106390009DF8200000069DF8211040EA01409DF87C
:1063A000221040EA01209DF823100843E86004F120
:1063B0001000C4B2286800140190686800140290AC
:1063C000A86800140390E868001404900198404302
:1063D000029901FB0100039901FB0100049901FBF3
:1063E000010ABAF1706F02DBBAF1885F22DDFDF7B6
:1063F0002BFC00203080401E94E721E0B8AAB38D2A
:10640000B4980D355D000000B8AAAAAAB088C3C52B
:10641000C700000009E3CA02AC010020D8B1B9F3FB
:106420008BA391B609B4D900DAB1B9F38BA391B6B5
:10643000DAB4DA00B6F9000040F48070308000BFB2
:106440003448807A00F0400020B305A9601C085C45
:10645000095D40EA012000B2A8F8000005A9E01C8F
:10646000095C05AAA01C105C41EA002000B2A8F853
:10647000020005A9601D095C201D105C41EA002096
:1064800000B2A8F80400A01DC4B2B6F9000040F0A4
:10649000080030801F48408900F4C07008B305A987
:1064A000601C085C095D40EA012000B2388005A943
:1064B000E01C095C05AAA01C105C41EA002000B2A7
:1064C000788005A9601D095C201D105C41EA002050
:1064D00000B2B880A01DC4B2B6F9000040F0700050
:1064E00030800C48807A00F0030018B105A9081923
:1064F000FFF7B4FE4846FDF706FF002012E701460D
:1065000004480160002070470146024841600020B5
:1065100070470000AC010020FBF76CFC4FF4E13049
:10652000FCF70EFA11A11648FCF7D4FAFCF7F4FBBD
:10653000C820FBF793FD13A11148FCF7CBFAD0203C
:10654000FBF7C1FE0446224612A10D48FCF7C2FA31
:10655000FDF774F8FDF786F86420FBF77FFD04E093
:106560000520FBF77BFDFDF7EBF8F9E7496E697451
:1065700020426C756520746F6F74682E2E0D0A00B2
:10658000004400404949432053746F702E2E0D0A79
:106590000000000049494320496E69742052657328
:1065A000203D2025640D0A00704700BFFEE700BFB4
:1065B000FEE700BFFEE700BFFEE770477047704789
:1065C000704710B54C1084EA530404D54042C1F121
:1065D000000138BF491E1B4204D55242C3F10003DB
:1065E00038BF5B1E00F0C6F814F0804F04D0404264
:1065F000C1F1000138BF491E14F0004F04D05242CF
:10660000C3F1000338BF5B1E10BD00000FB4044986
:1066100010B503AA029800F07DF910BC5DF814FBD8
:10662000380000202DE9F0410E460446002020628B
:106630002046E168884730B3252805D0D4E90121F8
:106640009047206A401CF2E7E1682046002788470F
:10665000050018D0A5F14100192802D820354FF4C3
:1066600000673246294620462760F9F79BFD40B176
:10667000012804D0F61D26F007060836D8E7361D97
:10668000D6E72846DAE7206ABDE8F0812DE9F04137
:106690000646002410687529314616A510D0AFF3C0
:1066A0000080002802DA404213A507E031688A071B
:1066B00001D512A502E0490704D511A5012401E086
:1066C000AFF3008000210A2206F1240709E0B0FBA5
:1066D000F2FCB0FBF2F302FB1C0030307854184699
:1066E000491C0028F3D123462A463046BDE8F04134
:1066F00000F0B7B8000000002D0000002B000000E3
:106700002000000040EA010310B59B070FD1042AC6
:106710000DD310C808C9121F9C42F8D020BA19BA6C
:10672000884201D9012010BD4FF0FF3010BD1AB1D1
:10673000D30703D0521C07E0002010BD10F8013B26
:1067400011F8014B1B1B07D110F8013B11F8014B4D
:106750001B1B01D1921EF1D1184610BD02F0FF03A0
:1067600043EA032242EA024200F0E8B87047704769
:106770007047704753EA020C00F069802DE9F04B36
:106780004FF00006002B1FBFB3FA83F503FA05F4A0
:1067900024FA05F65E4012BF1643B2FA82F502FAF9
:1067A00005F4C5F120051EBF22FA05FC44EA0C04DD
:1067B000203556EA044C4FEA144418BF641C4FF0CD
:1067C00000084FF00009904271EB030C39D3002907
:1067D00019BFB1FA81F701FA07F6B0FA80F700FAAB
:1067E00007F6C7F120071EBF20FA07FC46EA0C0691
:1067F0002037B6FBF4FCA7EB0507103F07F01F0B93
:10680000CBF120060CFA0BFB2CFA06F644BFB3467C
:106810000026202FA4BF5E464FF0000B5BEA060C5B
:1068200008BF4FF0010B19EB0B09ABFB027C48EBE7
:106830000608C01B06FB02CC0BFB03CC71EB0C0162
:10684000C1E70B46024641464846BDE8F08B13B50A
:106850004FF000004FF00001AFF30080BDE81C4096
:1068600070472DE9F0470D4699469246044600F1DF
:1068700024080168880604D5E06921F01001216030
:1068800000E00120A84201DD471B00E00027A169CC
:106890007A1902EB0900081AA0612078C00602D418
:1068A0002046AFF30080002608E0D4E901211AF861
:1068B00006009047206A401C761C20624E45F4DB9F
:1068C0002078C0060AD52046AFF3008006E0D4E960
:1068D000012130209047206A401C2062381EA7F119
:1068E0000107F4DC07E0D4E9012118F8050090471E
:1068F000206A401C2062281EA5F10105F3DC204619
:10690000AFF300802078000602D50220BDE8F087B2
:106910000120FBE7074B70B50D467B4400F033F8D0
:106920000446284600F042F810B14FF0FF3070BD29
:10693000204670BD23B6FFFF4FF000020429C0F0CF
:10694000128010F0030C00F03780CCF1040CBCF185
:10695000020F18BF00F8012BA8BF20F8022BA1EBF3
:106960000C0100F029B85FEAC17C24BF00F8012BBC
:1069700000F8012B48BF00F8012B704701694A1C41
:1069800002610878704700B58FB0CDE90131002170
:10699000059105497944CDE9031011466846FFF792
:1069A00041FE0FB000BD0000E5FFFFFF007B00F0DF
:1069B000800070474FF0000200B51346944696469B
:1069C000203922BFA0E80C50A0E80C50B1F1200102
:1069D000BFF4F7AF090728BFA0E80C5048BF0CC0B0
:1069E0005DF804EB890028BF40F8042B08BF70470E
:1069F00048BF20F8022B11F0804F18BF00F8012B80
:106A00007047000000487047BC0100207546FFF742
:106A1000F9FFAE4605006946534620F0070085465B
:106A200018B020B5F9F7E4FBBDE820404FF00006B0
:106A30004FF000074FF000084FF0000B21F0070166
:106A4000AC46ACE8C009ACE8C009ACE8C009ACE8A9
:106A5000C0098D46704710B50446AFF3008020464C
:106A6000BDE81040F9F7B0BB490050EAC12018BF9B
:106A700004204A0D18BF40F0010040F2FF72B2EB53
:106A8000515F08BF40F00200012808BF0520704791
:106A90002DE9F0414F1E00EBC7010446D1E900018A
:106AA00015461E4637F006020DD02A46334600F042
:106AB0005BFC7F1E04EBC703D3E9002300F04CFA14
:106AC00037F00602F1D1022F25D0042F13D0062F64
:106AD00018BFBDE8F0812A46334600F045FCD4E9F2
:106AE0000A2300F039FA2A46334600F03DFCD4E987
:106AF000082300F031FA2A46334600F035FCD4E989
:106B0000062300F029FA2A46334600F02DFCD4E98A
:106B1000042300F021FA2A46334600F025FCD4E98C
:106B2000022300F019FA2A46334600F01DFCD4E98E
:106B30000023BDE8F04100F00FBA012201F0E3B9F3
:106B400000F00ABA024A0020110701F0DCB9000087
:106B500001FDFFFF2DE9F84F04460D4621F00040EE
:106B600000917349814211DC7249884201DC06D1EF
:106B70002CB120462946BDE8F84FFFF7DEBF6E482E
:106B8000002DCCBF6D496E49BDE8F88F6D4981423B
:106B900011DD6D498142D8BF4FF0FF366DDD2046D3
:106BA0002946FFF761FF042808BFFFF7CBFF204607
:106BB0002946BDE8F88F6549654F25F000458142BB
:106BC00033DD6449814219DD002632464FF08043AF
:106BD0002046294600F0C0F980468A460122204618
:106BE000294601F090F900223B4600F0C7FC4246DE
:106BF000534600F061FA04460D463EE001260022AD
:106C0000BA463B462046294600F0A6F980460F4684
:106C1000002253462046294600F0B0FC42463B463F
:106C200000F04AFA04460D4627E04B4981421BDD3D
:106C3000DFF828A10226002253462046294600F00C
:106C400093FB00223B4600F087F980460F46002266
:106C500053462046294600F091FC42463B4600F050
:106C60002BFA04460D4608E0032622462B46002058
:106C70003B4900F021FA04460D4622462B461046B9
:106C8000194600F071FB8B46824602460B4600F027
:106C90006BFB07460246334888460B46062178447C
:106CA000FFF7F6FE52465B4600F05EFB82462E483A
:106CB0008B463A46434605217844FFF7E9FE3A46BB
:106CC000434600F051FB02460B46002E5046594603
:106CD0000CDA00F041F922462B4600F045FB01B0EA
:106CE00022462B46BDE8F04F00F03CBC00F034F9E2
:106CF00022462B4600F038FB1C4A7A4402EBC603BE
:106D0000D3E9002300F03AFC22462B4600F036FC83
:106D1000174A7A4402EBC603D3E9002300F022FCB1
:106D2000009A002AB8BF81F00041BDE8F88F00004A
:106D3000000010440000F07F182D4454FB21F93F5F
:106D4000FB21F9BF0000DC3F0000203E0000F33FC4
:106D50000000F03F0000E63F008003400000F83FE5
:106D60000000F0BFA61F0000641F0000021F00000B
:106D7000CA1E00002DE9F04D9446CCF1000423F02A
:106D800000464CEA0404524F46EAD4749A468846B8
:106D900021F00042BC4206D8454240EA050442EADE
:106DA000D474BC4204D9BDE8F04D6246FFF7C8BEBA
:106DB000AAF14055A5F17F6555EA0C040BD00224D9
:106DC00004EAAA74434DDFF810E144EAD87452EAA9
:106DD000000B04D00CE0BDE8F04DFFF7BBBE002C6B
:106DE00014BF012CBDE8F08D022C30D0032C32D022
:106DF00056EA0C0B0AD0BE4220D1BA4209D126F085
:106E0000804622F080423346114617E000291ADB03
:106E100025E0DFF8C8B0FB44002C04BFDBE900012B
:106E2000BDE8F08D012C02BFDBE9000181F00041DB
:106E3000BDE8F08D022C0AD0032C0CD0BA4212D13E
:106E4000B8F1000F0BDA23482549BDE8F08D28463C
:106E50002449BDE8F08D28467146BDE8F08D1D48F7
:106E60002149BDE8F08D921B12153C2AC4BF194878
:106E70001D490EDCBAF1000FBEBF12F13C0F00201D
:106E8000014606DB624600F017F921F00041FFF7EA
:106E900061FE002C08BFBDE8F08D012C04BF81F01D
:106EA0000041BDE8F08D114A114B022C07D000F0D3
:106EB00065FB2A46BDE8F04D0A4B00F05FBB00F0D1
:106EC0005DFB2A46BDE8F04D064B00F04BBB0000D1
:106ED0000000F07F182D4454FB2109C05E1E000005
:106EE000FB21F9BFFB210940FB21F93F075C14336B
:106EF00026A6A13C21F00042A2F16052B2F5801F0B
:106F000001F0004328BFD2F17F6C0BD95FEA001C6F
:106F100043EAC20242EB507018BF704728BF20F00E
:106F200001007047B2F5801FBCBF184670474FEA9A
:106F3000410C1CF5001F02D2084600F0FCBE70B5E3
:106F400000F0BCFA00000089FFF7F6BF4FF00040E8
:106F5000A0F580007047000010B591EA030F48BF0C
:106F600083F0004300F11283841A71EB030C05D205
:106F7000121943EB0C03001B61EB0C01DFF824E159
:106F80004FEA1154A4EB135C1EEA430F18BF9EEAAC
:106F9000445F73D023EA0E03DCF1200E21EA045192
:106FA00043F4801332D322FA0CFE10EB0E0023FAC6
:106FB0000CFE41EB0E01CCF1200E03FA0EFE10EB9D
:106FC0000E0051F10001B1F5801FCCF1200E32D23C
:106FD00001EB045112FA0EF2BDE8104058BF7047A1
:106FE000401C38BF5FEA420218BF7047002814BF38
:106FF00020F0010041F100014FEA410313F5001FA9
:1070000038BF7047A1F1C04100F0A6BA012A43EB96
:107010000302ACF1200CDCF11F0E32BF4FF0000E6A
:1070200023FA0CF310EB030041EB0451B4EB115FB6
:10703000D0D0A1EB045101F5801149085FEA30007E
:1070400001EB04510ED350F1000038BF12FA0EFECE
:1070500008D1BDE81040C9E7401C38BF5FEA4202D2
:10706000CAD1C3E7BDE810404FEA410313F5001F42
:1070700038BF7047A1F1C04100F06EBA9EEA445F8C
:1070800008D011EA5E0FBDE8104004BF01F00041D6
:1070900000207047BDE8104070B500F00FFA00BF47
:1070A00064FBBE3E0000E0FF02494FF0000000F02C
:1070B000F8BE00BF0000F87F2DE9C04130B4DFF812
:1070C000A0C23CEA111418BF3CEA131400F0EC8093
:1070D00081EA03051CEA111444EAD57418BF1CEABE
:1070E000131500F0C780A4EB05044FF0004545EAF6
:1070F000C12145EAC32341EA505143EA525304F106
:107100007F74994204F500344FEAC0204FEAC2224E
:1071100008BF904200F09C804FEA13650FF24016C2
:10712000765D4FEA134506FB05F7C7F1807706FB4E
:1071300007F74FEAD737A7FB03687642C8F58038D0
:10714000A7FB06CE38BFA8F1010807FB08E64FF001
:10715000000EA6FB028CE6FB03CEDCF1000CCEF1A8
:10716000004E38BFAEF1010EA6FB0C584FF00007E1
:107170004FF00005E6FB0E87A1FB08C6A0FB07CE7B
:1071800016EB0E0645F10005E1FB076515F1E04E33
:107190007EBFA4F580345FEA46066D4116F1800794
:1071A00045F100054FEA17274FEA066647EA0567EB
:1071B000A6F1DE46B6F1805F4FEA15251FD93846A5
:1071C00024F0010C05EBC471BCF1FE6F01EB0C1156
:1071D00002D8F0BCBDE8008124425CBF01F5801EEE
:1071E0009EEAC47F02D4F0BCBDE80081244238D4BA
:1071F000F0BCA1F1C041BDE8004100F0ADB94FEADB
:10720000D22242EA43524FEAD323A7FB02864FEA37
:10721000D02040EA415007FB03661EEA0E0F4FEAFA
:10722000D12105FB026658BFA6EB0056B6EB00560F
:107230004FEA520E4EEAC37E18EB0E0E56EB530E7B
:10724000BDD518EB02085E417F1C55F10005B6E77D
:107250004FF480154FF000074FF000064FF0000884
:10726000ADE7F0BC4FF0000001F1C04101F000417A
:10727000BDE8008111EA0C1F0CEA131500D00CE0E8
:1072800013EA0C1F00F025804FF00000F0BC81EAEB
:10729000030101F00041BDE80081F0BCBDE8004100
:1072A00081EA030100F058B9F0BCBDE8004170B5B7
:1072B00000F004F9097EFC3E00F007B881EA030102
:1072C0004FF0000001F00041704781EA030100F037
:1072D00043B9F0BCBDE800414FF0000021497047C0
:1072E000FFFDFBF9F7F5F4F2F0EEEDEBE9E8E6E48B
:1072F000E3E1E0DEDDDBDAD8D7D5D4D3D1D0CFCD12
:10730000CCCBCAC8C7C6C5C4C2C1C0BFBEBDBCBB4A
:10731000BAB9B8B7B6B5B4B3B2B1B0AFAEADACAB45
:10732000AAA9A8A8A7A6A5A4A3A3A2A1A09F9F9E1F
:107330009D9C9C9B9A9999989797969595949393D1
:10734000929191908F8F8E8E8D8C8C8B8B8A898968
:1073500088888787868585848483838282818180EB
:107360000000FF070000F87FDFF848C170B51CEA95
:10737000111E1EBF1CEA13159EEA0C0F95EA0C0F96
:1073800000F06F8081EA030423EA4C134EEAD47EB6
:1073900021EA4C1141F4801143F48013AE44A1FB67
:1073A000024CA0FB0365AEF17F7E361955EB0C0550
:1073B000A1FB034C4CF10003A0FB021C16EB0C06D6
:1073C000654153F10003094218BF46F0010613F46A
:1073D000007F0BD14FEA03314FEA0530340341EA15
:1073E000155140EA16506FF003020AE04FEAC3213C
:1073F0004FEAC520F40241EA555140EA56506FF079
:10740000020202EB2E4201EB025585EACE710AD050
:107410005FEA440C18BF24F0004450F1000041F131
:10742000000120EAD47040F2FE7C624500D270BDBB
:10743000A84214BF4FF080444FF04044002E08BFD4
:107440000024BEF1806FA8BFA1F1C041BDE870402B
:1074500080F282804FF0000001F1C04101F0004154
:1074600070479EEA0C0F0CEA131518BF95EA0C0F33
:1074700006D04FF0000081EA030E0EF0004170BD0F
:1074800000F01CF88900013E00F007B800F009B8D0
:107490004FEA430C5FEA5C5C08D081EA030100F02C
:1074A0005BB84FEA410C5FEA5C5CF6D14FF000003C
:1074B000014970470000FF070000F87F0EF1020E3F
:1074C0002EF0030E5EF8046B364205D4012A43EB1E
:1074D000030515F5001F12D8012841EB010C1CF51E
:1074E000001F0CD80ED14FEAD17C15F5001F0CEB14
:1074F0004C0C0CF1020C08BF4CEBD37C04E04FF0B9
:10750000080C01E04FEAD37C0CEB4C0526FA05F69B
:1075100006F00706B6F1040C06D20EEB860CBDE8A9
:1075200070404CF0010C6047DFE80CF0090B0202E0
:107530004FF000414FF00000A1F5002170BD194649
:107540001046012851EB010418BFD4F5001484BF84
:10755000002001F0004170BD0808A0F500114FEABD
:107560003101704791EA030F10B581F000413FF5FA
:10757000FBAC83F0004300F009B8000010B591EABD
:10758000030F48BF83F000433FF5EEAC841A71EB64
:10759000030C07D212198CF0004C43EB0C03001BB8
:1075A00061EB0C01DFF8A4E14FEA1154A4EB135C8A
:1075B0001EEA430F18BF9EEA445F00F0B08023EA42
:1075C0006E03524221EA0451C3EB6E0338BF5B1EC7
:1075D000DCF1200E25D322FA0CFE10EB0E0043FA4C
:1075E0000CFE41EB0E01CCF1200E03FA0EFE10EB67
:1075F0000E0051F10001CCF1200E29D412FA0EF246
:1076000001EB0451BDE8104058BF7047401C1CBF3F
:10761000B2F1004F704700280CBF491C20F0010058
:10762000704712EB020E43EB030218BF4FF0010E3E
:107630004EEA4202ACF1200CDCF11E0E54D943FAA2
:107640000CFE10EB0E0051F1FF31CCF11E0ED5D522
:107650000EF1010E12FA0EFE404141EB010101EB69
:10766000445C5FEA5C5C10D910EBDE7001EB045106
:1076700038BFBEF1004FBDE8104018BF704700286A
:107680000CBF491C20F00100704730D24FEAD42CC7
:1076900011F5001124F400641BD0B1FA81F20B3A09
:1076A000A41AA41ED2F12003914030FA03F3194327
:1076B000904001EBCC71002C01EB0451BDE810406F
:1076C000A8BF704701F1C0414FF0000001F0004138
:1076D0007047B0FA80F310FA03F100D110BDE41A3C
:1076E000173C4805C90AE4E701EB045110BD4910F5
:1076F00001EB0451BDE810404FEA300002E04FF0CA
:10770000000170474A0008BF0042F8D0B2F5001FE0
:1077100028BF704701F000414FF0000070479EEA1B
:10772000445F07D011EA5E0FBDE8104004BF00219E
:1077300000207047BDE8104070B5FFF7BFFE00BFE6
:1077400040DFF63E83F00041104670470000E0FF46
:1077500043004FEAD30C4FEA3C0C43401FBF4007A5
:107760000CF1605113F0FE4F70471CF0006F03D115
:1077700000200CF0004170470CF0004343EA5070C9
:1077800010B540EACC0000F090FA00BF0000009273
:107790004FEA0001FFF7E0BE4FF000414FF000005C
:1077A000A1F500217047000090EA010F48BF81F069
:1077B000004100F10883421A3CBF801A89184FEA41
:1077C000D0524FF07F4C1CEA410FA2EBD15318BFAF
:1077D0009CEA026F00F03B804FF0004C4CEA002026
:1077E0004CEA012121FA03FC10EB0C0C1ED202F131
:1077F000FF325FEA1C2040EBC25038BF70471CF0DC
:107800007F0F4FEA400C18BFBCF17F4F38BF704765
:10781000C3F12003994008BF20F00100BCF17F4F65
:1078200038BF7047A0F1C04000F085BA4FEA3C0075
:10783000000A40EBC25028BF1CF0FF0F4FEA400C7B
:10784000E6D018BFBCF17F4F38BF7047EAE79CEA2B
:10785000026F05D010EA5C0F08BF00F000407047CF
:1078600010B500F022FA00BF64FBBE3E401058BFC6
:10787000C0F14040491058BFC1F140418142EFF38F
:10788000008070474FF47F0C1CEAD0121EBF1CEA28
:10789000D11392EA0C0F93EA0C0F00F0858090EA66
:1078A000010F48BF42F4807240F4000C41F4000024
:1078B0002CF07F4120F07F4000B58142A2EB030213
:1078C0000FF2081CACEB504EC0F100009EF800E037
:1078D0004FEA4E0E00FB0EFC38BF49004FEA2C1C4D
:1078E00002F5FA020CFB0EF34FEACE1E4FEA112C02
:1078F0004FEAC1210EEB635E42EB22420EFB0CFC11
:107900004FEA1C5300FB03114FEA112C4FEA0131DF
:107910000EFB0CFC4FEADC4C00FB0C11C14228BFF3
:1079200009184CEB03335DF804EB10EB410143EB1A
:10793000C250B2F57C0F38BF704729D512F0F00F56
:107940001CBF00F1C04000F00040704700818283FE
:107950008485868788898B8C8D8E8F91929395965E
:1079600097999A9C9D9FA0A2A3A5A7A8AAACAEB0E8
:10797000B2B3B5B7B9BCBEC0C2C5C7C9CCCED1D4ED
:10798000D7D9DCDFE2E6E9ECF0F3F7FAFE0000001D
:107990004FEA400C0CF1807CBCF17E4F28BF704751
:1079A000B0F1C04000F0C7B990EA010F0CEAD11362
:1079B00048BF42F48072624538BF634507D213F472
:1079C0007F0F16D080EA010000F00040704710B52C
:1079D00000F06BF9097EFC3E00F005B880EA01007A
:1079E00000F00040704780EA010000F0004000F025
:1079F000A2B912F47F0F04BF0248704780EA010069
:107A000000F099B90000C07F50EA010C00F113802A
:107A10001CF5000F58BFBCF5000F01D48842704719
:107A200007D710F5000F58BF11F5000F15D4884285
:107A30007047894270471CF5000F04D5BCF5000F54
:107A4000F7D5814270474FF0807C1CEB400F38BF68
:107A50001CEB410F01D28142704710B500F025F9AF
:107A6000922449004FF000504FF08051FFF7FEBEC6
:107A700041000B0ED3F19E0208D950F400034FEAE7
:107A8000032323FA02F048BF4042704710B500F0CC
:107A90000CF900BF49922480002070476FF000422B
:107AA00082EA200070470000C10DD1F19E0206DB82
:107AB0004FEA002343F0004323FA02F070470042EC
:107AC00007D54FEA4001B1F1FE4F02D24FF000005E
:107AD000704710B500F0E9F8499224800020704703
:107AE0006FEA20007047000010F0004148BF40429C
:107AF000B0FA80F310FA03F2C3F19D030BD051EA00
:107B0000C35101EB1220530638BF704700F101004A
:107B100008BF20F001007047B0FA80F310FA03F2BA
:107B2000C3F19D030AD0D90501EB1220530638BFDB
:107B3000704700F1010008BF20F00100704700000D
:107B400050EA010C00F113801CF5000F58BFBCF582
:107B5000000F01D48842704707D710F5000F58BFB7
:107B600011F5000F15D488427047894270471CF503
:107B7000000F04D5BCF5000FF7D5814270474FF0D8
:107B8000807C1CEB400F38BF1CEB410F01D28142BF
:107B9000704710B500F089F8922449004FF000506A
:107BA0004FF08051FFF762BE4FF47F0C1CEAD012F9
:107BB0001EBF1CEAD11392EA0C0F93EA0C0F00F0DF
:107BC000478090EA010F48BF42F480724FF0004CAA
:107BD0004CEA00204CEA012102EB0302A0FB011356
:107BE000A2F50002002918BF43F001035B0028BF83
:107BF0004FEA330342EB22425FEA132C4CEBC250B4
:107C00002EBFBCEB436FB2F57C0F70474FEA036C9D
:107C1000BCF1004F08BF20F00100B2F57C0F38BF67
:107C200070470BD582F0FF0212F5803FC8BF704746
:107C300000F1C040D8BF00F00040704700F5000CD4
:107C40005FEA4C0C48BF7047B0F1C04000F073B819
:107C500090EA010F0CEAD11348BF42F480726245EA
:107C600038BF634504D280EA010000F0004070474D
:107C700010B500F01AF800BF8900013E00F007B807
:107C800000F009B85FEA410C5FEA1C6C08D080EA9A
:107C9000010000F050B85FEA400C5FEA1C6CF6D1BE
:107CA0004FF00040A0F5800070470EF1020E2EF05C
:107CB000030E5EF8044B244204D44FEA4102B2F1B1
:107CC0007F4F11D84FEA4003B3F17F4F0CD80ED14C
:107CD0004FEAD07CB2F17F4F0CEB4C0C0CF1020C54
:107CE00008BF4CEBD17C04E04FF0080C01E04FEAF8
:107CF000D17C0CEB4C0324FA03F404F00704B4F138
:107D0000040C06D20EEB840CBDE810404CF0010CC4
:107D10006047DFE80CF0070802024FF00040A0F5D2
:107D2000800010BD0846420018BFD2F1807288BFA3
:107D300000F0004010BDFF2141EAD050C00570475F
:107D400051EA000C00F113801CF5000F58BFBCF580
:107D5000000F01D48142704707D711F5000F58BFBB
:107D600010F5000F15D481427047894270471CF509
:107D7000000F04D5BCF5000FF7D5884270474FF0CF
:107D8000807C1CEB410F38BF1CEB400F01D28842B6
:107D9000704780EA010081EA000180EA0100FFF7F4
:107DA000F8BE80F0004090EA010F7FF504AD81F04D
:107DB000004100F008B8000090EA010F48BF81F0D0
:107DC00000413FF5F8AC421A04D882F00042A0EB23
:107DD000020011444FEAD0524FF07F4C1CEA410F91
:107DE000A2EBD15318BF9CEA026F4AD04FF0004C6F
:107DF0004CEA00204CEA012121FA03FCB0EB0C0C08
:107E00000FD412F0FE0F36D05FEA4C001DD50012E1
:107E100040EBC25038BF70471CF03F0F18BF70478F
:107E20000BE0A2F101025FEA1C2040EBC25038BF18
:107E300070471CF07F0F18BF7047C3F120039940B3
:107E400014BF401E20F00100704780084FEA122343
:107E500008BF7047B0FA80FCA2EB0C02CCF1280CF2
:107E600060FA0CF093EA122F04BF00EBC250704787
:107E70004FEAC3707047130A5FEADC1008BF70470F
:107E8000F6E79CEA026F04D010EA5C0F08BF0020FE
:107E9000704710B5FFF709FF40DFF63E81F0004064
:107EA00070470CF00F03092B08BF082000F0598021
:107EB0000A2B0BD0082B18BF704708BF1CF0400FCF
:107EC0000AD04FF000004FF0000170471CF0400F47
:107ED00018BF4FF0004070471CF0100F08D020F082
:107EE000704300F07F4242EAD3014FEA437070478B
:107EF00000F0604021F07F4242EA000201F07F4042
:107F000040EA727070474FF0FF0C4CF4E06C1CEAD2
:107F100011531CBF9CEA030C9445C2BFDA4201EB2B
:107F200002517047002B0DD0BCF1000F0FD0002A7A
:107F300001F00041A4BF41F0E04141F07F614FF00A
:107F40000000704701F000414FF00000704750EA18
:107F500001334FF09B0C18BF4CF0806C7FF4A4A849
:107F600070471CF4801F11D01CF4E02F03D06FEA7F
:107F7000CC31490070474FF04050EFF3008222F0BF
:107F8000704242EA000282F3008870474FF000001E
:107F9000704700006800000476005401F7FD0001FE
:107FA00075191A0C6A231B1C1F207274433B41383D
:107FB000393A6B6C376F06246D6E700083000000D9
:107FC00000080000000100183200050000002041F8
:107FD0000000D242295C0F3E9A99993E3333733F99
:107FE000295C0F3E00007000000000240000000229
:107FF0000003000000650054FFEF0000FA80000B52
:1080000012820001030C30C30E8C8CE914D540029F
:1080100013710F8E3883F8833000F883258EF88330
:108020003000F883FFFFFFFF0FFEA9D624000400F5
:108030001A8279A10000003CFFFF00000010000040
:1080400038836FA2003E03304000000002CAE309FB
:108050003E80000020000000000000004000000002
:1080600060000000000C0000000C186E000006927A
:108070000A16C0DFFFFF0256FD8CD377FFE1C496DE
:10808000E0C5BEAA00000000FFFF0B2B0000165742
:10809000000003594000000000001DFA00026C1DA2
:1080A000000000003FFFDFEB003EB3B6000D22787A
:1080B00000002F3C00000000001942B5000039A26A
:1080C0000000B365D90E9FC91DCF4C3430000000AD
:1080D000500000003BB67AE80064000000C80000D1
:1080E00000000000100000001000FA921000225E54
:1080F000000D229F0001000000320000FF4600003A
:1081000063D400001000000004D6000004CC00007E
:1081100004CC0000000010720000004000000000CD
:10812000000000000006000200050007000000003B
:10813000006400000000000000000005000500646D
:1081400000200000000000000000000000004000CF
:108150000000030000000032F8980000FF650000F6
:10816000830F0000FF9BFC000000000000000000E7
:1081700000000000000000000000000000000000FF
:1081800000000000000000000000000000000000EF
:108190000000100040000000000000060000B26A6D
:1081A000000200000001FB830068000000D9FC0011
:1081B0007CF1FF830000000000650000006403E81C
:1081C00000640028000000250000000016A0000048
:1081D0000000100000001000002F0000000001F45B
:1081E0000000100000280000FFFF4581FFFFFA7229
:1081F0000000000000000000004400050005BAC6B1
:10820000004778A200000001000000000000060006
:10821000000000140000254D002F706D000005AE19
:10822000000C02D000000000000000000000000070
:1082300000000000001B0000000000000000000023
:1082400000000000006400000008000000000000C2
:10825000000000000000000000000000000000001E
:10826000000000000000000000000000000000000E
:1082700000000000000000000000000000000000FE
:1082800000000000000000000000000000000000EE
:1082900000000000000000000000000000000000DE
:1082A00000000000001B00000000000000000000B3
:1082B000000E000E00000AC700040000000000329B
:1082C000FFFFFF9C00000B2B0000000200000001DC
:1082D00000000064FFE50000000000000000000056
:1082E000000000000000000100000000000100008C
:1082F00000000000000180000001800000018000FB
:10830000002426D30000000000000000000600103A
:108310000096003C0000000000000000000000008B
:10832000000000000C0A4E68CDCF7709501667593F
:10833000C619CE820000000000000000000000000E
:1083400000000000000000000000000017D78400BB
:10835000030000000000000000000000C7938F9D94
:108360001E1B1C190000000000000000000000009F
:10837000000000000000000000000000020318855B
:1083800000004000000000030000000300000000A7
:10839000000000004000000000000000000000009D
:1083A00000000000000000000000000000000000CD
:1083B00000000000000000000000000000000000BD
:1083C0000000000000000000677DDF7E72902E55E7
:1083D0004CF6E688000000000000000000000000ED
:1083E00000000000D8DCB4B8B0D8B9ABF3F8FAB3E9
:1083F000B7BB8E9EAEF132F51BF1B4B8B08097F1E9
:10840000A9DFDFDFAADFDFDFF2AAC5CDC7A90CC96C
:108410002C97F1A989264666B28999A92D557DB078
:10842000B08AA896365676F1BAA3B4B280C0B8A87E
:108430009711B28398BAA3F0240844106418B2B913
:10844000B49883F1A329557DBAB5B1A38393F00005
:108450002850F5B2B6AA839328547CF1B9A382932D
:1084600061BAA2DADEDFDB819AB9AEF5606870F13D
:10847000DABAA2DFD9BAA2FAB9A38292DB31BAA2E0
:10848000D9BAA2F8DF85A4D0C1BBAD83C2C5C7B835
:10849000A2DFDFDFBAA0DFDFDFD8D8F1B8AAB38D63
:1084A000B4980D355DB2B6BAAF8C96198F9FA70EF2
:1084B000161EB49AB8AA872C547CBAA4B08AB69176
:1084C000325676B28494A4C808CDD8B8B4B0F19925
:1084D00082A82D557D98A80E161EA22C547C92A41D
:1084E000F02C5078F184A898C4CDFCD80DDBA8FC02
:1084F0002DF3D9BAA6F8DABAA6DED8BAB2B68696FD
:10850000A6D0F3C841DAA6C8F8D8B0B4B882A89209
:10851000F52C548898F135D9F418D8F1A2D0F8F98F
:10852000A884D9C7DFF8F883C5DADF69DF83C1D84B
:10853000F40114F1A8824EA884F311D182F5D992E6
:10854000289788F109F41C1CD884A8F3C0F9D1D964
:108550009782F129F40DD8F3F9F9D1D982F4C20345
:10856000D8DEDF1AD8F1A2FAF9A88498D9C7DFF8C3
:10857000F8F883C7DADF69DFF883C3D8F40114F1B0
:1085800098A8822EA884F311D182F5D992509788A9
:10859000F109F41CD884A8F3C0F8F9D1D99782F175
:1085A00049F40DD8F3F9F9D1D982F4C403D8DEDF48
:1085B000D8F1AD8898CCA809F9D98292A8F57CF1B8
:1085C000883ACF944A6E98DB6931DAADF2DEF9D899
:1085D0008795A8F221D1DAA5F9F417D9F1AE8ED09A
:1085E000C0C3AE82C684C3A88595C8A588F2C0F171
:1085F000F4010EF18E9EA8C63E56F554F18872F431
:108600000115F19845856EF58E9E0488F142985AC1
:108610008E9E068869F4011CF1981E1108D0F5049D
:10862000F11E970202983625DBF9D985A5F3C1DA48
:1086300085A5F3DFD88595A8F309DAA5FAD8829243
:10864000A8F578F1881A849F26889821DAF41DF31A
:10865000D8879F39D1AFD9DFDFFBF9F40CF3D8FA13
:10866000D0F8DAF9F9D0DFD9F9D8F40BD8F3879F2D
:1086700039D1AFD9DFDFF41DF3D8FAFCA869F9F9D5
:10868000AFD0DADEFAD9F88F9FA8F1CCF398DB45AA
:10869000D9AFDFD0F8D8F18F9FA8CAF38809DAAF35
:1086A0008FCBF8D8F2AD978D0CD9A5DFF9BAA6F328
:1086B000FAF412F2D8950DD1D9BAA6F3FADAA5F2E6
:1086C000C1BAA6F3DFD8F1BAB2B68696A6D0CAF37D
:1086D00049DAA6CBF8D8B0B4B8D8AD84F2C0DFF18F
:1086E0008FCBC3A8B2B68696C8C1CBC3F3B0B4884B
:1086F00098A821DB718D9D71859521D9ADF2FAD8AD
:108700008597A828D9F408D8F28D29DAF405D9F28A
:1087100085A4C2F2D8A88D9401D1D9F411F2D887DA
:1087200021D8F40AD8F28498A8C801D1D9F411D874
:10873000F3A4C8BBAFD0F2DEF8F8F8F8F8F8F8F810
:10874000D8F1B8F6B5B9B08A95A3DE3CA3D9F8D86C
:108750005CA3D9F8D87CA3D9F8D8F8F9D1A5D9DF8A
:10876000DAFAD8B18530F7D9DED8F830ADDADED80C
:10877000F2B48C99A32D557DA083DFDFDFB591A0E6
:10878000F629D9FBD8A0FC29D9FAD8A0D051D9F81C
:10879000D8FC51D9F9D879D9FBD8A0D0FC79D9FA2D
:1087A000D8A1F9F9F9F9F9A0DADFDFDFD8A1F8F8F3
:1087B000F8F8F8ACDEF8ADDE8393AC2C547CF1A86D
:1087C000DFDFDFF69D2CDAA0DFD9FADB2DF8D8A8A1
:1087D00050DAA0D0DED9D0F8F8F8DB55F8D8A87870
:1087E000DAA0D0DFD9D0FAF8F8F8F8DB7DF8D89C19
:1087F000A88CF530DB38D9D0DEDFA0D0DEDFD8A8FA
:1088000048DB58D9DFD0DEA0DFD0DED8A868DB7027
:10881000D9DFDFA0DFDFD8F1A888902C547C98A89E
:10882000D05C38D1DAF2AE8CDFF9D8B087A8C1C1FC
:10883000B188A8C6F9F9DA36D8A8F9DA36D8A8F98D
:10884000DA36D8A8F9DA36D8A8F9DA36D8F78D9D0D
:10885000ADF818DAF2AEDFD8F7ADFA30D9A4DEF908
:10886000D8F2AEDEFAF983A7D9C3C5C7F1889BA7B2
:108870007AADF7DEDFA4F8849408A797F300AEF290
:108880009819A488C6A39488F632DFF28393DB0993
:10889000D9F2AADFD8D8AEF8F9D1DAF3A4DEA7F17D
:1088A000889B7AD8F38494AE19F9DAAAF1DFD8A8B4
:1088B00081C0C3C5C7A39283F628ADDED9F8D8A37B
:1088C00050ADD9F8D8A378ADD9F8D8F8F9D1A1DA54
:1088D000DEC3C5C7D8A18194F818F2B089ACC3C56E
:1088E000C7F1D8B8B4B09786A8319B069907AB9763
:1088F00028889BF00C201440B0B4B8F0A88A9A28BD
:108900005078B79BA8295179247059446938644834
:1089100031F1BBAB88002C547CF0B38BB8A8042891
:108920005078F1B088B49726A85998BBABB38B02A6
:10893000264666B0B8F08A9CA82951798B295179CE
:108940008A2470598B2058718A4469388B39406861
:108950008A6448318B30496088F1AC002C547CF03B
:108960008CA804285078F1889726A85998AC8C02D6
:10897000264666F0899CA8295179247059446938A3
:10898000644831A98809205970AB11384069A81989
:108990003148608CA83C415C207C00F187981986A6
:1089A000A86E767EA999882D557DD8B1B5B9A3DF7B
:1089B000DFDFAED0DFAAD0DEF2ABF8F9D9B087C4E2
:1089C000AAF1DFDFBBAFDFDFB9D8B1F1A3978E60CB
:1089D000DFB084F2C8F8F9D9DED89385F14AB183C3
:1089E000A308B5839A0810B79F10D8F1B0BAAEB0FB
:1089F0008AC2B2B68E9EF1FBD9F41DD8F9D90CF11A
:108A0000D8F8F8AD61D9AEFBD8F40CF1D8F8F8ADD0
:108A100019D9AEFBDFD8F416F1D8F8AD8D61D9F4D1
:108A2000F4ACF59C9C8DDF2BBAB6AEFAF8F40BD8FB
:108A3000F1AED0F8AD51DAAEFAF8F1D8B9B1B6A3CB
:108A4000839C08B9B1839AB5AAC0FD3083B79F1043
:108A5000B58B93F20202D1ABDADED8F1B080BAABBB
:108A6000C0C3B284C1C3D8B1B9F38BA391B609B462
:108A7000D9ABDEB0879CB9A3DDF1B38B8B8B8B8B2D
:108A8000B087A3A3A3A3B28BB69BF2A3A3A3A3A374
:108A9000A3A3A3A3A3F1B087B59AA3F39BA3A3DCDD
:108AA000BAACDFB9A3A3A3A3A3A3A3A3A3A3A3A324
:108AB000A3A3A3A3D8D8D8BBB3B7F1AAF9DAFFD937
:108AC000809AAA28B48098A720B79787A86688F0CC
:108AD0007951F1902C870CA781976293F0717160A6
:108AE00085940129517990A5F1284C6C870C951833
:108AF0008578A38390284C6C886CD8F3A28200F20E
:108B000010A8921980A2F2D926D8F188A84DD94888
:108B1000D896A83980D93CD89580A839A68698D906
:108B20002CDA87A72CD8A8899519A980D938D8A874
:108B30008939A980DA3CD8A82EA83990D90CD8A8B0
:108B4000953198D90CD8A809D9FFD801DAFFD89562
:108B500039A9DA26FFD890A80D8999A81080982104
:108B6000DA2ED88999A83180DA2ED8A88696318055
:108B7000DA2ED8A8873180DA2ED8A88292F34180E5
:108B8000F1D92ED8A882F31980F1D92ED882ACF36E
:108B9000C0A28022F1A62EA72EA92298A829DAAC7D
:108BA000DEFFD8A2F22AF1A92E8292A8F23180A685
:108BB00096F1D900AC8C9C0C30ACDED0DEFFD88CAA
:108BC0009CACD010ACDE8092A2F24C82A8F1CAF22A
:108BD00035F19688A6D900D8F1FF0000000000000A
:108BE0004FBB610567ACDD3F182D4454FB21E93FC5
:108BF0009BF681D20B73EF3F182D4454FB21F93FB4
:108C0000E2652F227F2B7A3C075C143326A6813C39
:108C1000BDCBF07A8807703C075C143326A6913CE4
:108C2000C4EB98999999C9BF711623FEC671BCBF50
:108C30006D9A74AFF2B0B3BF9AFDDE522DDEADBFB8
:108C40002F6C6A2C44B4A2BF0D5555555555D53FD0
:108C5000FF8300922449C23F6E204CC5CD45B73FEB
:108C6000513DD0A0660DB13FEB0D76244B7BA93F63
:108C700011DA22E33AAD903F00000000000000004E
:108C800050726F647563742049442072656164207A
:108C90006173203020696E64696361746573206458
:108CA00065766963652069732065697468657220FB
:108CB000696E636F6D70617469626C65206F72209C
:108CC000616E204D5055333035302E0D0A000000B6
:108CD000F08C000800000020180100006C01000862
:108CE000088E00081801002008070000880100080D
:108CF00000A24A040000000000000000010203047A
:108D00000607080900000000010203040102030431
:108D10000607080902040608000000000000000021
:108D20000000000000000000000000000000000043
:108D30000000000000000000000000000000000033
:108D400000000000000000004600000000000000DD
:108D50000000000000000000000000000000000013
:108D60000000000000000000000000000000000003
:108D700001000000000000000000000000000000F2
:108D800000000000000000000000000000000000E3
:108D900000000000000000000000000000000000D3
:108DA00000000000000000000000000000000000C3
:108DB0000000000000000000000000000000803FF4
:108DC000000000000000000000000000FF000000A4
:108DD000FF0000000100000000000000A07F00086C
:108DE000947F000800000000000000000000000068
:108DF0000000000000000000000000000000000073
:088E000000000000BC7F000827
:0400000508000131BD
:00000001FF
